:2000000028140020E9000000F1000000F300000000000000000000000000000000000000B7
:20002000000000000000000000000000FB0000000000000000000000FF00000001010000C4
:20004000030100000501000007010000090100000B0100000D0100000F0100001101000048
:20006000130100001501000017010000190100001B0100001D0100001F01000021010000A8
:20008000230100002501000027010000290100002B0100002D0100002F0100003101000008
:2000A000330100003501000037010000390100003B0100003D0100003F0100004101000068
:2000C000EF3BE8FF03B40148019001BD89FF00200448854600F070F800480047C90600004B
:2000E000C046C046281400201648804716480047FEE7FEE7FEE7FEE7FEE7FEE7FEE7FEE7A6
:20010000FEE7FEE7FEE7FEE7FEE7FEE7FEE7FEE7FEE7FEE7FEE7FEE7FEE7FEE7FEE7FEE78F
:20012000FEE7FEE7FEE7FEE7FEE7FEE7FEE7FEE7FEE7FEE7FEE7FEE7FEE7FEE7FEE7FEE76F
:20014000FEE7000095040000D100000030B50B46014600202022012409E00D46D5409D421C
:2001600005D31D469540491B2546954040191546521E002DF1DC30BDD2B201E00270401C8D
:20018000491EFBD270470022F6E710B513460A4604461946FFF7F0FF204610BD30B5044617
:2001A0000020034600E05B1C934203D2E05CCD5C401BF8D030BD0000064C0125064E05E0AF
:2001C000E36807CC2B430C3C98471034B442F7D3FFF782FF240B0000540B0000FFB581B07E
:2001E00004460D460020012C03D140262E43304306E0002C00D103E0022C01D1C0263043D8
:20020000012A06D1049E760010273E430643F0B206E0002A00D103E0022A01D13026304396
:20022000134E307076788027BE43114F7E70012C08D1FF2100BF0E4EB3781E460E40334642
:200240008B42F8D10A4E76784027BE43084F7E70012A0BD10026009603E000BF009E761C80
:200260000096FF276937009EBE42F6D905B0F0BD0004024070B5034614460020002B01D128
:20028000C0B202E005468035E8B2012902D1051DE8B206E0022903D105460835E8B200E0D0
:2002A000C0B2012C02D1851CE8B200E0C0B2084DA870AD7801263543054EB570002201E093
:2002C00000BF521C7D252D01AA42F9D970BD0000000C024070B50024244800792021084031
:2002E000002801D0224D3FE000F046F805462148007880210840002836D01E488078084060
:20030000002801D01A4D02E000F036F80546194880780007840F022C01DBAD0804E0012C6F
:2003200001D16D0800E000BF124880788007C00F002801D02D0101E00C2045430D480078A6
:200340004007840F002C02D1601CC4B207E0032C03D1601C4006040E01E06006040E214654
:200360002846FFF7F3FE0546284670BD0004024000127A00000C024000B5C0229178F82268
:2003800011401C4A12781143EA2923D00ADC0A46E03A130000F0CEF80A181C20242A2A2AA9
:2003A0002A161A2AED291FD004DCEB2916D0EC291CD117E0F02903D0F82917D10E4817E09F
:2003C0000E4815E00E4813E00E4811E00E480FE00E480DE00E480BE00E4809E00E4807E0FD
:2003E0000E4805E00E4803E00E4801E00D4800BF00BF00BD201C02400090D003006CDC0297
:200400000048E80100366E010024F400001BB70000127A00808D5B0000093D00C0C62D002F
:2004200080841E0040420F0010B501231A4600211846FFF7D3FE012211461046FFF71AFF9B
:20044000FFF740FE034800F01DF902480249086010BD00000090D0031800002010B500F0FD
:2004600063F810BD1A20084908722B2048723C2088724D20C8727F20044909680860AC20BC
:20048000034948707047000000040240140000200010024010B580201B4948711A201A49B6
:2004A000203908722B2048723C2088724D20C872002016494860FFF70DFF15490860002058
:2004C000C0431449086014490860144814490860114903221202891848600F4989188860B1
:2004E0000D498918C8600C49891808610A498918486109498918886107498918C861AC201F
:200500000849487010BD00002004024000B001401800002080E200E000E100E0C0C0C0C073
:2005200000E400E000100240AC200149487070470010024030B47446641E2578641CAB42A4
:2005400004D3635D5B00E31830BC18471D46F8E702E008C8121F08C1002AFAD17047704712
:20056000002001E001C1121F002AFBD170470000F8B510484568876800F066F80024E443A0
:2005800009E0287860400006800D0B490858210A484004466D1C38467F1E0028F1D1E44339
:2005A00004480068A04201D0012000E0002006463046F8BD1C0000202800002070B500256E
:2005C00061246402202221461548FFF7E7FD002823D120222146403111484030FFF7DEFD80
:2005E00000281AD12022A1180D482030FFF7D6FD002812D120222146603109486030FFF763
:20060000CDFD002809D110222146803104488030FFF7C4FD002800D100E00125284670BD77
:20062000940A0000014600200A06FF231B020B401B021A43FF231B040B401B0A1A430B0E7A
:200640001A4310467047000010B5002113E0084608220AE0C307DB0F002B04D04308074CA4
:200660006340184600E04008521E002AF2D18B00034CE050491CFF29E9D910BD2083B8ED86
:200680002800002010B5044603492046FFF75EFD0249087010BD000040420F0000000020BF
:2006A00070B505460E462C460BE0204600F0EBF8A004800C002801D1FFF7D0FE012080024F
:2006C0002418B442F1D370BD10B5012464073748374908603748384908603848384908606A
:2006E000334800680068401C00284ED0304800680068314909680968884246D030480068A9
:200700004068002841D12A4909680868FFF78AFF2C490860264909684868FFF783FF2949CD
:200720004860234909688868FFF77CFF25498860084680686114401803218903884224D20A
:20074000FFF73CFF002820D1FFF712FF00281CD1FFF788FEFFF768FE00F03AF815490C319E
:200760001448FFF79DFF12480C210268114800F0CEF800BFBFF34F8F13481449C860BFF3AA
:200780004F8F00BF00BF00BFFDE772B6012109042046FFF7F8FC01210903086880F3088812
:2007A00000BF48688047002010BD000020C0000008000020001450000C000020001050001E
:2007C000100000201C0000200400FA0500ED00E0F0B5FFB0FFB083B01A48416800910321E7
:2007E000890301200003FFF75BFF01252D0315488068A9104018401E860A00271CE0FF221B
:200800000121890201A8FFF7B7FC002406E0B80201190098415C01AA1155641C0120800292
:200820008442F4D301AA0146284600F070F8012080022D187F1C761E002EE0D17FB07FB01F
:2008400003B0F0BD1C000020014672B608208C4AD060F120106255205060AA2090600020DD
:20086000C043086000BF86480068C007C00F0028F9D00120824A10600020D060F020106262
:2008800062B600207047014672B610207C4AD060F120106255205060AA2090600020C0434F
:2008A000086000BF76480068C007C00F0028F9D00120734A10600020D060F020106262B62C
:2008C0000020704770B503461D46F1206C4E3062002415E072B6AA20694E70605520B060FC
:2008E00010782870521C6D1C62B600BF64480068C007C00F0028F9D00120614E3060641C8F
:200900008C42E7D3F0205E4E3062002070BDF7B55C4B9D4406460F4600215B48684481618D
:20092000012104918802874207D95748684481618069554B28339D44F0BD029600240EE084
:20094000029800785049694448610298401C02904869FF2801D000200490601C84B2BC4201
:20096000EED3049800280AD0484849490860464868443946426A3046FFF7A4FF6FE0B00A11
:200980004500F119681C4002814202D90120039001E000200390B10A89020191B105890D38
:2009A0000091039800280ED0002408E00198007805A908550198411C0191601C84B2324829
:2009C0008442F3DB0EE0002408E00198007805A908550198411C0191601C84B20120800290
:2009E0008442F2DB002410E027486844406A02780099081905A90A5423486844406A411C2D
:200A0000214868444162601C84B2BC42ECD30398002815D01D481E4908606802FFF733FF41
:200A20001A481B490860691C4802FFF72CFF174817490860680205AA1349FFF743FF0EE0D6
:200A40001248134908606802FFF71DFF0F4810490860680205AA01218902FFF733FF0A48A4
:200A60006844806965E730B50446002304E025781570641C521C5B1C8B42F8D330BD000053
:200A800000000240E4F7FFFF00080000CDAB341204000020484A5F3735305F544654000077
:200AA0000000000000000000000000000000000000000000484A59422D3735303054465422
:200AC00000000000000000000000000000000000000000004241543332413237394B4D3629
:200AE000344642000000000000000000000000000000000043414E5F5354445F4348305FA5
:200B00003530304B627073000000000000000000000000008907000081070000DF070000B2
:200B200000000000540B0000000000201C00000050050000700B000000FF0020D00000005B
:200B400050050000700B00001C0000200C1400006005000000000000000000000000000004
:200B60000000000000000000C00000000000000040203149087100BF00BF00BF00BF00BFA7
:200B80002D480079802108400028F9D0704710202949087100BF00BF00BF00BF00BF264892
:200BA0000079202108400028F9D070472348007880210840002810D020480078400840004F
:200BC0001E49087000BF00BF00BF00BF00BF1B480078802108400028F9D1002016490871CD
:200BE00000BF00BF00BF00BF00BF13480079602108400028F9D170471048007801210843B7
:200C00000E49087000BF00BF00BF00BF00BF0B480078802108400028F9D0002006490871BD
:200C200000BF00BF00BF00BF00BF03480079402108400028F9D1704700040240000C02404F
:20100000785F0020E9100000F1100000F310000000000000000000000000000000000000DC
:20102000000000000000000000000000FB1000000000000000000000FF1000002162000013
:201040009D420000014300004943000091430000D94300002144000069440000B1440000EA
:20106000F9440000414500008D450000D9450000ED450000394600004D46000061460000D2
:20108000AD460000114700007D470000E947000055480000C1480000D548000021490000E4
:2010A0006D490000B5490000014A00006D4A0000814A0000954A0000014B00006D4B0000CC
:2010C000EF3BE8FF03B40148019001BD89FF00200448854600F094F900480047E589000077
:2010E000C046C046785F00201648804716480047FEE7FEE7FEE7FEE7FEE7FEE7FEE7FEE7FB
:20110000FEE7FEE7FEE7FEE7FEE7FEE7FEE7FEE7FEE7FEE7FEE7FEE7FEE7FEE7FEE7FEE77F
:20112000FEE7FEE7FEE7FEE7FEE7FEE7FEE7FEE7FEE7FEE7FEE7FEE7FEE7FEE7FEE7FEE75F
:20114000FEE7000081650000D110000030B50B46014600202022012409E00D46D5409D42AF
:2011600005D31D469540491B2546954040191546521E002DF1DC30BD70B5002425460028D4
:2011800001DA01244042002901DA01254942FFF7DDFFAC4200D04042002C00D0494270BD52
:2011A00003460B439B0703D009E008C9121F08C0042AFAD203E00B780370401C491C521E6C
:2011C000F9D27047D2B201E00270401C491EFBD270470022F6E710B513460A460446194659
:2011E000FFF7F0FF204610BD30B504460020034600E05B1C934203D2E05CCD5C401BF8D0B6
:2012000030BD0321001D401E037812021A43491EF9D510467047034603220870000A491CBF
:20122000521EFAD518467047024670B54A40D30FDB0740002DD04A002AD0010E140E0002EB
:2012400012020919400A520A8418E50104465443000A120A2E045043A4194219200CC54318
:20126000AA18120C0125AD03521C521912047F39240400D0521C104301D44000491EC2B268
:201280000C06C0092018401C4008802A02D003E0002070BD40084000002900DA00201843E5
:2012A00070BD70B502464A40D50F40004A00ED0740085208002814D0002A12D0C40DD30D3D
:2012C00041020120C0055202490A520AE41A091812187D34914201D3641C00E04900002C6C
:2012E00001DA002070BD0023914201D3891A0343400849000028F7D100290AD0914202D1E9
:201300000121C90705E0914201D2012101E00121C943E005C018401900F030F870BD10B5FF
:2013200000229623114600F031F810BDC20FD207400040080BD0C10D0723DB01C918400291
:201340000905400A1143C20840071143704700200146704710B5002904DB0124E407404248
:201360008C412146002B04DB1C460123DB075242A341994200D1904210BD0000002904DAFD
:20138000401C490001D140084000704770B40024050C05D11024000402D1002921D011240E
:2013A000050E01D100020834050F01D10001241D850F01D18000A41C002801DB4000641C78
:2013C000002908D020252E1B0D46F540A14000D001212943084301061B1B000ADB1D02D556
:2013E000002070BC7047DB05181880180029F8DA401C4900F5D170BC400840007047000071
:20140000064C0125064E05E0E36807CC2B430C3C98471034B442F7D3FFF75EFED4930000AB
:201420000494000070B58C180578401C6B075B0F01D10378401C2A1106D10278401C03E022
:2014400006780E70401C491C5B1EF9D12B0705D40023521E0DD40B70491CFAE70378401C75
:20146000CB1A921C03E01D780D70491C5B1C521EF9D5A142D8D3002070BD0000F0B5FFB09B
:20148000FFB083B003208003224908600121C9042320400307F07EFA1F480078002802D133
:2014A000312005F095FD23267603E82700242AE0FF220121890201A8FFF784FE002507E05A
:2014C000A002401913490968085C01A948556D1C012080028542F3D301AA0146304607F081
:2014E0008CFB012080023618641C7F1E0A480078002808D16006400E002804D1002C02D0DD
:20150000312005F065FD002FD2D17FB07FB003B0F0BD0000BC020020C0020020F0B5FFB07F
:20152000FFB083B0232040031749086001460320800307F02FFA0325AD03E82600271DE064
:20154000FF220121890201A8FFF73CFE002407E0B80200190C490968085C01A90855641C55
:20156000012080028442F3D301AA0146284607F044FB012080022D187F1C761E002EDFD1B1
:201580007FB07FB003B0F0BDBC02002010B500210720400204F0F2F90021194804F0EEF924
:2015A0000021184804F0EAF900211648801E04F0E5F90A2001F0A2F80121114804F0DEF9E9
:2015C0000F2001F09BF801210720400204F0D6F91E2001F093F80121FF20063004F0CEF91E
:2015E0000A2001F08BF801210648801E04F0C6F90F2001F083F80121024804F0BFF910BD0C
:20160000030400000507000010B50146002000BF0EE04200124B9A5A124B9A4206D24200F8
:201620000F4B9A5A521843000D4CE252421CD0B20328EEDB0C4A12680C4B1B689A4204D2F2
:20164000094A12685218084B1A60094A1268094B9A4204D2064A12685218054B1A6010BDE8
:201660001C000020102700003000002034000020040000208813000010B502469000074BA5
:20168000C018405C002802D00320C04310BD01209300024C1B1958540020F7E7441A00208B
:2016A00010B50024FFF772FF00203349087000BF07E000206100314A505231490855601C2F
:2016C000C4B2032CF5DB00202E4908802E490860012080022D4908804B20C00048800846B5
:2016E0000079FC21884380302849087108460079800880000871002048710846807900097E
:201700000001401C887108468079F021884350301E4988710846C07980088000C87108465A
:20172000C0790C2188431949C8710846C079302188431649C8710846C079C0218843134913
:20174000C8710C2008811420488104208881A020C8810882182048820D4848610020487600
:2017600007200876084604F023FD0A4804F052FD04F0F2FA10BD0000220000201C000020A2
:201780002300002026000020280000201013002000400D032C13002010B509490B6809688B
:2017A000491C074C21600749C8542146096801221203914202D300212246116010BD000005
:2017C0000000002010030020F0B589B006A908A802F000FB0546089803906D48046808994C
:2017E000069888427ED208988442FBD2C8E00698A04203D30698001B079004E00898001B11
:201800000699401807900398002803D00398401E039000E0B8E0285DEB2871D10898401EC8
:20182000611C0840285C9028F7D10798062868D90898401EA11C08402E5C36020898401E0E
:20184000E11C0840285C06430898401E211D0840285C05900598000205900898401E611D29
:201860000840285C0599084305900598C04380B2B0425DD1089886425AD80798B04256D3D8
:201880000898401EA11D08402F5C3F020898401EE11D0840285C07433F020898401E491CC2
:2018A0000840285C07433F020898401E491C0840285C07430020C04332460A3A0090089849
:2018C000401E491C0840029001462846089B00F039FC04900498B84214D1089883B2304694
:2018E0000A3800E051E082B20898401E21460A31084080B201460290284603F031FC06E0FA
:201900002FE02DE023480068401C224908600020285500220898401E611C08402A54A019F0
:201920000899491E084004461948046028E02BE019480068401C1849086000202855002288
:201940000898401E611C08402A540898401E10490968491C08400E490860084604680FE069
:2019600012E0079802280AD30898401E08490968491C0840064908600846046800E003E02E
:201980000698844200D032E700BF09B0F0BD0000FC020020CC020020D002002070B501466B
:2019A000002058256D5A1C2635402B4658256B5204251D40002D04D008251D40002D00D053
:2019C000012004251D40002D2DD053256D5C10263540002D27D01A4DA94201D1194A00E0BF
:2019E000194A00240CE001E00125D581D589ED07ED0F002DF8D10225D5811032651CECB2F5
:201A0000102CF0DBFF2650256E5252256D5C002D02D0002652256E540126F60350256E5272
:201A2000FF2607366E5208251D40002D06D052256D5C002D02D0002652256E5470BD00002C
:201A4000005404400055044000590440582211527047014600205322525C10231A40002AE3
:201A600008D05322525C0C231A409210032A18D1032016E05422525A0123DB031A40002A69
:201A80000ED05322525C0C231A409210032A05D05322525C9207920F032A01D1022000E0BA
:201AA000012070470246002058239B5A0B40002B01D0012000E00020704710B5002A0AD08E
:201AC00056231B5A0C0223435624235256231B5A8B43235209E056231B5A0C02A34356243F
:201AE000235256231B5A0B43235210BDF8B504460D46012700263448844203D10121022001
:201B000000F026FA2878401EA0702088FF210131084320802088400840002080A878401E74
:201B2000C1B25A20015568790007000CE97909020843A97908435C210853288981B240202D
:201B40000153A868C000C10C42200153A88981B244200153E868C000C10C46200153288A79
:201B600081B2482001532869C000C10C4A200153A88A81B24C2001536869C000C10C4E20A9
:201B800001535020005B297909020843502108535020005B297988435021085300E0761CEC
:201BA0005020005B4007400F2979884202D007488642F4D15020005B4007400F29798842DD
:201BC00000D000273846F8BD00540440FFFF00000146144AC889C007C00F00280AD0012096
:201BE000C88100E0521EC889C007C00F002801D0002AF7D1C889C007C00F00280FD1022069
:201C0000C8810420C881487A400840004872487A3823984348720020487201207047002086
:201C2000FCE70000FFFF00000246507A012318435072507A0B78DB0018435072087A012880
:201C400008D1888850814868000C0123DB031843908108E0087A002805D150814868800037
:201C6000204B18409081487A012804D1507A40231843507206E0487A002803D1507A4023B5
:201C800098435072087D002804D0507A80231843507203E0507A8023984350720878002807
:201CA00011D1C87A1072087B1070487B5070887B9070CB7BD370087C10714B7C5371887CD8
:201CC0009071CB7CD371887A002803D00120C002D08101E00820D081FF200130D08101202B
:201CE00070470000FC1F0000002904D0427A80231A43427203E0427A80239A43427270471B
:201D000030B5024600200F4B5024A45A0D022C435025AC525024A45A8C43AC5200E05B1E21
:201D20005024A45A6407640F8C4201D0002BF6D15024A45A6407640F002C01D0002000E075
:201D4000012030BDFFFF0000F0B587B006460C460027002006906020875BF807C00F0028C8
:201D600002D001216020815355E0FF20000238400005000F06902B48864204D106980001F4
:201D80002949451806E02948864203D106980001274945180420E881A8890121C903084021
:201DA000002809D0012069460872A889C004C00869890843019007E0002069460872A889EC
:201DC0001C49084080100190287A6946C872002003E02A5C03A90A54401C6946C97A814206
:201DE000F7DCA088172801DB0020A08061881822514322460832881818226946FFF7D0F9EC
:201E00006188481C1721FFF7B7F96180A088401CA0806020875B022038400028A5D007B0C2
:201E2000F0BD000000540440005504400058044000590440FC1F000010B502461D4BD089A2
:201E4000C007C00F00280AD00120D08100E05B1ED089C007C00F002801D0002BF7D1D089EB
:201E6000C007C00F002801D0002010BD507A012420435072507A3824A0435072C87A107243
:201E8000487A00280FD1087B1070487B5070887B9070CC7BD470087C10714C7C5471887CCE
:201EA0009071CC7CD471FF200130D0814000D081107ADAE7FFFF0000FFB581B004460D4697
:201EC0000020012C03D140262E43304306E0002C00D103E0022C01D1C0263043012A06D176
:201EE000049E760010273E430643F0B206E0002A00D103E0022A01D130263043134E30709B
:201F000076788027BE43114F7E70012C08D1FF2100BF0E4EB3781E460E4033468B42F8D1B0
:201F20000A4E76784027BE43084F7E70012A0BD10026009603E000BF009E761C0096FF275D
:201F40006937009EBE42F6D905B0F0BD00040240002905D0054A12780243044B1A7004E0F3
:201F6000024A12788243014B1A70704720040240002905D0054AD27E0243044BDA7604E06E
:201F8000024AD27E8243014BDA7670470008024070B5034614460020002B01D1C0B202E00A
:201FA00005468035E8B2012902D1051DE8B206E0022903D105460835E8B200E0C0B2012C48
:201FC00002D1851CE8B200E0C0B2084DA870AD7801263543054EB570002201E000BF521CC8
:201FE0007D252D01AA42F9D970BD0000000C024070B500242448007920210840002801D028
:20200000224D3FE000F046F805462148007880210840002836D01E4880780840002801D022
:202020001A4D02E000F036F80546194880780007840F022C01DBAD0804E0012C01D16D08E4
:2020400000E000BF124880788007C00F002801D02D0101E00C2045430D4800784007840FD6
:20206000002C02D1601CC4B207E0032C03D1601C4006040E01E06006040E21462846FFF78D
:2020800065F80546284670BD0004024000127A00000C024000B5C0229178F82211401C4A6C
:2020A00012781143EA2923D00ADC0A46E03A130006F078FB0A181C20242A2A2A2A161A2AEC
:2020C000ED291FD004DCEB2916D0EC291CD117E0F02903D0F82917D10E4817E00E4815E09B
:2020E0000E4813E00E4811E00E480FE00E480DE00E480BE00E4809E00E4807E00E4805E0D0
:202100000E4803E00E4801E00D4800BF00BF00BD201C02400090D003006CDC020048E80163
:2021200000366E010024F400001BB70000127A00808D5B0000093D00C0C62D0080841E0001
:2021400040420F00FFB50C460021099800BF16E066185F1E3E40009FBE5D3606704000252D
:202160000AE0C60FF607002E04D04600064F7E40304600E040006D1C082DF2DB491C9142EF
:20218000E6DB04B0F0BD0000B71DC10408B501460A78CB781A436B461A704A7852108B78FC
:2021A0005B001A43D3B26A4653708A7892104B789B001A43D3B26A469370CA78D2100B7831
:2021C000DB001A43D3B26A46D370127810066A465278120410436A469278120210436A46FB
:2021E000D278104308BD000010B50446002006F0E5FB022841D121480078002802D101203F
:202200001E4908701D48007801281FD11B484078401C1A49487021465A20FEF797FF17498B
:202220004978884229D800201449487008468078401C8870084680780A2803D300208870DD
:2022400002200870002006F0E5FB16E00B480078022812D109484078401C0849487021464B
:202260007D20C000FEF772FF04494978884204D800200249487006F0CDFB10BD7C0000209D
:2022800000B587B0002168460171042141710A48029001460391049105910848069001A8C1
:2022A00006F0D6FB00F05AF800F00CF80021044803F064FB07B000BDFFFFFF1F352300007A
:2022C0000205000010B5184818494860002008720120087000204872012088721448FFF74F
:2022E00077FC12491248FFF79FFC01211048FFF7FBFC0D485E300D49486000200872012022
:202300000870002048720120887209481030FFF75FFC064906481030FFF786FC01210448AB
:202320001030FFF7E1FC10BD810700006C1700201055044010B5044607496068884204D024
:2023400005495E396068884205D1E17A22460C32606800F09DFC10BDDF07000000B587B03F
:202360000E4802900021684601730171417381730821C173002004E0002204A90A54411C2D
:20238000C8B26946C97B8142F6DC0548FFF720FC01A90348FFF748FC07B000BD89070000A9
:2023A0000055044030B587B00446002520680290A1796846C173617941730021017301714E
:2023C00000BF05E020460830415D04A841556D1C6846C07BA842F5D8084902984018002847
:2023E00008D101A90648FFF727FD0021029800F0D7FB00E000BF00BF07B030BD77F8FFFF06
:2024000000550440FEB504460E460020019003208003844203D023204003844202D1FF3490
:20242000FF34023461204002844202D02348844240D1204606F06CFA002838D100962048A5
:20244000009E864230D2E01FFF38FA380290029800F0CAF907460020C0431A490860254627
:202460000EE028781749097848400006800D1649085814490968090A4840124908606D1C5E
:202480000098411E00910028EBD10E480068C0430C49086008460068B84202D1002001901E
:2024A0000AE00120019007E00220019004E00420019001E0032001900198FEBD00620400FE
:2024C000009E0300B0020020908F000010B50124640701F08DFC09480068094988420AD1EB
:2024E00006484068002808D161132046FEF771FE02F0E8FB01E002F0BBFB10BDB4020020A6
:20250000A55A7AA730B5FFB0FFB083B01C48008A1B49498A884205DB1948008A1849498A37
:20252000401A84B2002C26D0FF220121890201A8FEF748FE00250CE01148418A1430405C22
:2025400001A948550E48408A401C0D494882681C85B2A542F0DB21460948143006F088F9B8
:20256000074901AA0868214606F047FB044800680019034908607FB07FB003B030BD0000D2
:20258000A42D002010B500202C4908702C49087001F02EFC2B4840682B49884204D02948D2
:2025A00040682A49884210D1264840682649884202D101202149087002202549087005F033
:2025C0006FFF002006F0D4F837E01E4840682149884203D101201A4908702EE0194840686B
:2025E0001D49884224D100F0D1F81C4880680121C90488421CD219480068612149028842AA
:2026000016D11648416823204003FFF7FBFE00280ED1FEF783FF00F08BF8114A51681068DA
:20262000FFF7F0FE002803D106F0A2F804F0CAFD05F036FF01200649087010BD99020020D5
:20264000C0020020B4020020A33A7AA7A88A7AA7970200208BB86336A55AA55AC8310020C5
:20266000BC31002010B5014600200A781306180E00064A781304FF242404234018438A7876
:202680001302241223401843CA78104310BD014600200A06FF231B020B401B021A43FF2332
:2026A0001B040B401B0A1A430B0E1A431046704710B50024312004F08BFC0E4A516810686D
:2026C000FFF7A0FE002812D1FEF7D8FE00F05EF8312004F07DFC0848416823204003FFF717
:2026E00091FE002801D1012402E0002400E00124204610BDBC310020C831002010B50446B9
:202700000020094908600948046001E003F0E4FA05480068054909688842F7D30020024905
:2027200008600249086010BD300000203400002010B5134800F058F8124908601048001D75
:2027400000F052F80F494860084600686121490288420FD10B4840680B49884202D90020FE
:20276000C04304E0074840686121490240180549886003E00020C0430249886010BD00001A
:2027800004C00000BC310020003E070010B5124800F02AF8114908600F48001D00F024F8B0
:2027A0000E494860084600686121490288420ED10A4840680A49884202D90020C04303E0F6
:2027C00006484068074940180449886003E00020C0430249886010BD04600400C83100209F
:2027E000009E03000062040038B50446002000906A460421204606F0ACFA0098FFF747FF40
:202800000090009838BD02460020082905D30A2903D80C2A26D1012024E00E2903D8102A7E
:2028200020D101201EE0122903D8142A1AD1012018E0162903D8182A14D1012012E01E2995
:2028400003D8202A0ED101200CE02E2903D8302A08D1012006E03E2903D8402A02D101205B
:2028600000E00020704701460020022903D3082901D8012010E00C290BD0102909D01429BF
:2028800007D0182905D0202903D0302901D0402901D1022000E00020704710B500F034FF09
:2028A00000F00CF900F062FB00F002F810BD0000FEB5002455480078912852D100F0F4F87B
:2028C0000128FAD1524800685249086008460079F021884320304F4908710846007900092B
:2028E00000014A49097A0907090F0843494908714648807A401E4549887208460189C088B5
:20290000401E81422ED2082142484030017100BF0EE03E4841883E48801D415C3D48401D63
:2029200001553A484088401C38494880601CC4B2072CEED33748066840300779002406E085
:202940003448001D005D69460855601CC4B2082CF6D3012000F0ECFD6A463946304600F0F7
:20296000CFF952E029480189C088401E814242D12648007925498978401AC5B2072D2FDC80
:20298000681CC1B223484030017100240EE01F4841881F48801D415C1E48401D01551B4894
:2029A0004088401C19494880601CC4B2AC42EEDB1848066840300779002406E01548001DDE
:2029C000005D69460855601CC4B2082CF6D3012000F0AEFD6A463946304600F091F914E0D0
:2029E00000F0E2FD00200949087009490868092100F0CAF909E000F0D7FD002003490870EE
:202A000003490868092100F0BFF9FEBDE42200207C2200204C1D00202049097800293CD0E1
:202A20001E498978482251431D4A51581D4A116000200CE01949897848225143184A8918D8
:202A4000091D0A5C1749091D0A54411CC8B21349897848225143124A891840310979814221
:202A6000E8DC0E498978482251430D4A891840310A790C4940310A7101224A710749097860
:202A8000491E064A117011468978491C917011468978082901D3002191707047B81C002016
:202AA000781A0020041D00200349487B012802D10021014A51737047F422002010B53348BB
:202AC0004068002861D13148007B030005F06AFE07590512212E3D4A59002D4800780028E5
:202AE00007D000202A4908702A490868012100F04BF947E026480078002809D00020244920
:202B0000087025498A8801230868891D00F04CF938E01F480078002807D000201C4908705B
:202B20001C490868022100F02FF92BE018480078002809D000201649087017498A8809230C
:202B40000868891D00F030F91CE011480078002807D000200E4908700E490868092100F0AA
:202B600013F90FE00A480078002809D000200849087009498A8803230868891D00F014F909
:202B800000E000BF00BF00F00FFD10BDF4220020E42200207C220020941D0020704700006C
:202BA00070B504460D4636480068A04267D1002D65D134480078222852D004DC202841D057
:202BC00021285AD145E0902802D0912855D115E02C48C08801280AD100202A49087000F043
:202BE000E3FC29490868002100F0CEF805E0032000F09EFCA020234908703FE021480089F6
:202C0000401C2049088108460089C98888420AD100201C49087000F0C7FC1B4908680021F4
:202C200000F0B2F80DE01748807A002806D000F0BBFC1449087B00F05BFC02E0032000F0F3
:202C400077FC1BE0062000F073FC11200D49087014E0062000F06CFC11200A4908700DE027
:202C600000200849087000F09FFC08498A8809230868891D00F098F800E000BF00BF70BD30
:202C8000BC1C0020E42200207C220020941D002070B50346184C2478082C2CD2164C6478A9
:202CA00048256C43154D2B5100200AE0155C124C647848267443114EA419241D2554441C0A
:202CC000E0B28842F2DB0C4C647848256C430B4D641940342171084C2478641C064D2C7041
:202CE0002C466478641C6C702C466478082C02D30025014C657070BDB81C0020781A0020B9
:202D0000F0B587B007460D4616461D480760002406E031781A48001D0155761C601CC4B203
:202D2000AC42F6DB2C4605E0AA211548001D0155601CC4B2082CF7DB11480068029008216E
:202D40006846C1730021417301730171002406E00B48001D015D04A80155601CC4B2082CD6
:202D6000F6DB01A90748FFF767F800210298FFF717FF012102484030017107B0F0BD0000BB
:202D8000BC1C00200055044070B504460D462946204604F037F970BD70B504460D46294689
:202DA000204604F03DF970BDF8B504460D4616461F463B4632462946204604F032F9F8BDA9
:202DC000F0B585B006460F46154665480078002804D009213046FFF7D7FFBEE0002D01D0F4
:202DE000602D04D909213046FFF7CEFFB5E05D4806608580002405E0395D5A48801D01552D
:202E0000601C84B2AC42F7DB00205549487008468580FF2088727F200873084680880828BE
:202E200031D20120C880084680884880012008814C4800684C49086008460079F0218843C2
:202E4000494908710846007900090001444909790907090F08434449087141480079401CB0
:202E6000C1B2414840300171002407E03D48801D015D3D48401D0155601C84B23848808877
:202E8000A042F3DC4CE00721681CFEF75FF9002907D0072128460830FEF758F93049C88087
:202EA00005E00721681CFEF751F92D49C88006202B494880012008812A4800682A490860C3
:202EC00008460079F02188431030274908710846007900090001224989880905090F084368
:202EE0002149087108468088FF21090288431C4989880902FF221202114008431A498880E6
:202F00000821194840300171002407E01548801D015D1548801D0155601C84B2062CF5D3E6
:202F20001148006803901048403000790290002406E00D48001D005D69460855601C84B2D3
:202F4000082CF6D3012000F0F3FA9020044908706A4602990398FFF7D3FE05B0F0BD0000F2
:202F6000E42200207C2200204C1D002010B5FFF753FD14484079002823D01248403800795E
:202F80000009002806D0012807D002280AD0032810D10CE000F010FA0FE000F0C5F800F0A8
:202FA00011FB0AE000F010F800F00CFB05E000F06BF902E0FFF7F2FD00BF00BF0021014844
:202FC000417110BD441D002010B55348007811281AD15248006852498842F9D14F480079B4
:202FE0000007000F4C49097A0907090F88420CD000204949087000F0D7FA4A498A8804231E
:203000000868891DFFF7D0FE84E043480089401C414908810846807A401E88720846008978
:20302000C988884249DA3D4840300079082822D03A48403000790C281DD0384840300079CD
:20304000102818D0354840300079142813D033484030007918280ED03048403000792028A0
:2030600009D02E4840300079302804D02B484030007940284ED12948403000792649897B3C
:20308000884247D100240EE02448401D015D224842882448801D81541F484088401C1E4911
:2030A0004880601CC4B21D4840300079401EA042EAD8062000F03CFA2CE0174880881649E8
:2030C0004988411A154840300079814222DA00240EE01248401D015D0F4842881148801D81
:2030E0008154601CC4B20C484088401C0A49488009484088084989888842EADB00200649FD
:20310000087000F051FA07498A8800230868891DFFF74AFE10BD0000E4220020041D0020EF
:2031200081070000941D002070B500255248007880210840802871D05048006850498842A5
:203140006CD14E4840300079082867D34B4840300079082822D04948403000790C281DD010
:20316000464840300079102818D0444840300079142813D041484030007918280ED03F480D
:2031800040300079202809D03C4840300079302804D03A484030007940286CD13748007984
:2031A0000407240F240235488088000A0443334840300079401EA0425DD801202E494870AC
:2031C0002E4840300079801E48802C48403000798873084684800120088100208872C87282
:2031E000264A40321279511E234A9288501CFDF7ADFF002913D02048818820484030007992
:2032000008181D49C8801D4A40321279511E1A4AD088FDF79BFF1849C8800BE02BE0174AC3
:2032200040321279511E144A9288501CFDF78EFF1149C88011480068124908600846848045
:20324000002507E00D48801D415D0E48801D4155681CC5B2094840300079801EA842F1D8C3
:20326000042000F065F9102003490870054A91881068FFF791FD70BDE4220020041D0020F0
:2032800081070000941D002010B547480078A02807D045480078912803D043480078A1280D
:2032A0000ED142480068424988420AD0414908680921FFF769FD00F077F900203A49087013
:2032C00071E03A484030007903280AD2394908680921FFF759FD00F067F900203249087060
:2032E00061E0324800790007000F002804D001282DD002284BD136E02B484078002800D0E3
:2033000050E02A484079002803D101202649487003E0264840792449887223480078912801
:203320000BD022488079002804D0204880791E49087302E001201C49087391201A490870A1
:2033400000F032F91849087B00F0D2F82AE016484078002800D025E0A120134908700320DF
:2033600000F0E6F81EE010484078002800D019E00D480078A02809D10E4908680821FFF72B
:2033800003FD00F011F90020074908700AE0094908680521FFF7F8FC00F006F90020024935
:2033A000087000BF00BF10BDE4220020041D0020810700007C22002070B50024484800784C
:2033C0008021084080284FD04648056844480078002802D04448854246D14249403108795D
:2033E000FFF741FA0546002D08D0012D04D13D4800790407240F01E03A48447939484030FC
:203400000079A0426BDD012D2FD1364800790007000F002863D0334840300079401EA042CF
:203420005DD330480068314908602E4800790007000F8880002407E02A48401D015D2B48E2
:20344000801D0155601CC4B228488088A042F3DC00202349087000F0A7F824498A88002329
:203460000868891DFFF7A0FC39E0022D37D11D4800790007000F002831D1082C2FDB194897
:2034800040300179A01C814229D31649403108792146FFF7B8F9002821D012480068134931
:2034A0000860104840798880012408E00D48401D025D601E0D49891D0A54601CC4B20B4850
:2034C0008088A042F2DA00200549087000F06CF806498A8800230868891DFFF765FC70BDDE
:2034E000E4220020041D002081070000941D00207F2807D8411CC8B27D21C90041430B4A6F
:2035000091600EE0F12808D3F92806D80107090F64225143054A916003E07D218902034A06
:2035200091600221014A517370470000F422002000B5030005F036F90729050B11171D23F7
:2035400029000121144A11731449516022E00221114A1173114951601CE003210E4A117325
:203560000F49516016E004210B4A11730D49516010E00521084A1173002151600AE0062178
:20358000054A11730649516004E00021024A1173516000BF00BF00BDF422002070110100DF
:2035A000F0490200282300000020014908737047F4220020024909880918014A1180704723
:2035C000F42200207CB500244A480078102849D149488088494988420AD949480079000919
:2035E0000001801C4649087122204249087008E043480079000900014149087120203D4922
:20360000087040483E49086008460079F021884330303B490871084640793649897A0846E4
:2036200037494871084680790020887103213448403001714038056840300679002406E091
:203640002F48001D005D69460855601CC4B2082CF6D30220FFF76CFF6A4631462846FFF770
:203660004FFB46E023480078112842D12148807A00283ED11F48407800283AD11D4988725F
:203680001F480079000900011D4908712020194908701C481A49086008460079F021884375
:2036A000303017490871084640791249897A0846134948710846807900208871032110482D
:2036C000403001714038056840300679002406E00B48001D005D69460855601CC4B2082C2B
:2036E000F6D30220FFF724FF6A4631462846FFF707FB7CBDE4220020941D0020E204000023
:203700004C1D002089070000244A118852888A4242D0224A52888A4204DA204A52888A1AF9
:2037200090B207E01D4A52880023DB439A1A521C521890B2194A5180127B002A10D0174AE4
:203740005268002A0CD0154A5268824205D9134A5268121A114B5A6002E000220F4B5A607D
:203760000E4A527B022A17D10C4A9268002A0CD00A4A9268824205D9084A9268121A074B00
:203780009A6002E00022054B9A60044A9268002A02D10122014B5A7370470000F422002073
:2037A00010B5002006490870401E06490860064908608321C9000548FDF70BFD10BD00000E
:2037C000A9020020AC020020B0020020A42D0020F8B50023002500950024002200BF95E089
:2037E00001259D40ACB20D8825400095009DA54270D11A468D79012D0DD1464D03263602AE
:20380000AD192D5C012696403543424E03273F02F61935540CE03F4D03263602AD192D5C29
:2038200001269640B5433B4E03273F02F6193554CD78002D4FD1374D60352D5CCE78002E5F
:2038400001D1012600E000269640B543314E603635548D78002D2ED12E4D19267601AD19D5
:203860002D5C8E78002E01D1012600E000269640B543284E19277F01F61935540D79002D3D
:203880000ED1244D50352D5C0E79002E01D1012600E000269640B5431E4E5036355424E0C9
:2038A0001C4D50352D5C0E799640F6B23543194E5036355419E0174D19267601AD192D5C3C
:2038C0008E789640F6B23543124E19277F01F61935540AE018E00F4D60352D5CCE789640BC
:2038E000F6B235430B4E603635544D79012D0AD1084D30352D5C01269640F6B23543054EAE
:203900003036355400E000BF5D1CABB2082B00DA66E7F8BD00000440FFB581B00746154663
:203920001E4600243846029900F01CF8002802D0012005B0F0BD00240CE00A206043084937
:20394000085CB04204D12946204600F047F803E0601C84B2232CF0D300BF0020E9E70000E2
:20396000808D00000246002A03D1402901DD01207047032A03D1022901DD0120F8E7042A9D
:2039800003D1202901DD0120F2E7052A03D1202901DD0120ECE70C2A03D1102901DD0120D2
:2039A000E6E70D2A05D1012903DD402901DA0120DEE70E2A03D1202901D10120D8E70020D2
:2039C000D6E70000014A11547047000090000440014A1154704700008000044070B5024657
:2039E00000205EE10A235343B04C1B195B1C440004191B579B1C002B3DD00A235343AB4C82
:203A00001B195B1C440004191B195B78082B33D10A235343A54C1B195B1C440004191B5D24
:203A2000A34CA44D6419E35C5C0864000A2353439E4D5B195B1C450045195B5D9C4D9D4E5A
:203A4000AD19EC540A235343984C1B195B1C440004191B5D964C35466419E35C0224A34310
:203A60000A245443914D6419641C45004519645D8F4DAD192B5562E00A2353438B4C1B1910
:203A80005B1C440004191B195B78092B33D10A235343864C1B195B1C440004191B5D844C26
:203AA000844D6419E35C4024A3430A2454437F4D6419641C45004519645D7D4D7D4EAD19E2
:203AC0002B550A235343794C1B195B1C440004191B5D774C35466419E35C8024A3430A24A8
:203AE0005443724D6419641C45004519645D704DAD192B5523E00A2353436C4C1B195B1CE3
:203B0000440004191B5D6A4C6A4D6419E35C0A245443664D6419641C450045196419657831
:203B20000124AC40A3430A245443604D6419641C45004519645D5E4D5E4EAD192B550A23F1
:203B400053435A4C1B195B1C440004191B199B788B427DD10A235343544C1B195B1C440069
:203B600004191B195B78082B33D10A2353434F4C1B195B1C440004191B5D4D4C4D4D641958
:203B8000E35C012423430A245443484D6419641C45004519645D464D464EAD192B550A2306
:203BA0005343424C1B195B1C440004191B5D404C35466419E35C022423430A2454433B4DC1
:203BC0006419641C45004519645D394DAD192B5564E00A235343354C1B195B1C4400041924
:203BE0001B195B78092B34D10A2353432F4C1B195B1C440004191B5D2D4C2E4D6419E35C13
:203C0000402423430A245443284D6419641C45004519645D264D274EAD192B550A2353434E
:203C2000224C1B195B1C440004191B5D204C35466419E35C8024A3430A2454431B4D6419BB
:203C4000641C45004519645D194DAD192B5525E025E00A235343154C1B195B1C440004199A
:203C60001B5D134C134D6419E35C0A2454430F4D6419641C45004519641965780124AC4025
:203C80002343DCB20A235343084D5B195B1C450045195B5D064D074EAD19EC5404E0431CE1
:203CA000D8B2032800D29DE600BF70BD808D000000000440750800000149086070470000D7
:203CC0000C03002002480068401C01490860704708030020F3B581B0064600200E4908600F
:203CE00000F01EF8044600F01BF805462F1B3046029900F0F2FF00900AE000F011F805462C
:203D00002F1B06480068002802D004480068804700988742F1D3FEBD080300200C030020F4
:203D2000014800687047000008030020034A12680260034A12680A60704700003C00002083
:203D40004000002070B505461D480068002835D11C48007800280DD101201A490870002397
:203D60001A461946284601F05FF9FF20F5301649088023E000231A461946012001F054F95E
:203D80000446022C07D110480088401E80B20E490880002812D1022C0DD020200849086075
:203DA000022D03D100200949086001E00748046000200749086000200249087070BD0000AA
:203DC0005000002074000020760000205800002068000020024601200003106002480068BB
:203DE000086002487047000000000020100300200348044A01681160001D016851607047A6
:203E000000105000B402002010B50446032C00D110BD002C01D0012C7ED10021084601F0B7
:203E200041FD0021012001F03DFD0021022001F039FD8021032001F035FD0021042001F050
:203E400031FD8021052001F02DFD8021062001F029FD8021480001F025FD8021FF20023087
:203E600001F020FD8021FF20033001F01BFD0021FF20043001F016FD0021FF20053001F05A
:203E800011FD8121FF20063001F00CFD0021FF20073001F007FD0021FF20083001F002FD4F
:203EA00000210120400201F0FDFC0021F24801F0F9FC0021F048401C01F0F4FC0021EE4866
:203EC000801C01F0EFFC00218120800001F0EAFC0021E948001D01F0E5FC0021E648401D64
:203EE00001F0E0FC0021E448801D01F0DBFC80210320000201F0D6FC0021E04801F0D2FCB2
:203F00008021C80001F0CEFC0021DD4801F0CAFC0021DB48401C00E097E001F0C3FC802138
:203F2000D748801C01F0BEFC00210520000201F0B9FC8021D34801F0B5FC8121D148401CB8
:203F400001F0B0FC0021CF48801C01F0ABFC8121CC48C01C01F0A6FC0021CA48001D01F0F2
:203F6000A1FC80210320400201F09CFC8021C64801F098FC8021C448401C01F093FC8021B7
:203F8000C148801C01F08EFC80210720000201F089FC8021BD4801F085FC8021BB48401CA9
:203FA00001F080FC8021B948801C01F07BFC8021B648C01C01F076FC8021B448001D01F065
:203FC00071FC0021B148401D01F06CFC8021AF48801D01F067FC81210320800201F062FC85
:203FE0008021AB4801F05EFC0021A948401C01F059FC8021A648801C01F054FC0021A448B5
:20400000C01C01F04FFC00210D20000201F04AFC8021A04801F046FC80219E48401C01F071
:2040200041FC80210720400201F03CFC00219948FB3001F037FC8021974801F033FC80217E
:204040009548401C01F02EFC14E10021084601F029FC0021012001F025FC0021022001F00A
:2040600021FC8021032001F01DFC0021042001F019FC8021052001F015FC8021062001F08A
:2040800011FC8021480001F00DFC8021FF20023001F008FC8021FF20033001F003FC002145
:2040A000FF20043001F0FEFB0021FF20053001F0F9FB8021FF20063001F0F4FB0021FF2053
:2040C000073001F0EFFB0021FF20083001F0EAFB00210120400201F0E5FB0021664801F06B
:2040E000E1FB00216448401C01F0DCFB00216248801C01F0D7FB00218120800001F0D2FBC9
:2041000000215D48001D01F0CDFB00215A48401D01F0C8FB00215848801D01F0C3FB802181
:204120000320000201F0BEFB0021544801F0BAFB8021C80001F0B6FB0021514801F0B2FBEA
:2041400000214F48401C01F0ADFB80214C48801C01F0A8FB00210520000201F0A3FB8121D4
:20416000484801F09FFB81214648401C01F09AFB00214448801C01F095FB80214148C01C42
:2041800001F090FB00213F48001D01F08BFB81210320400201F086FB81213B4801F082FB5B
:2041A00081213948401C01F07DFB81213648801C01F078FB80210720000201F073FB80212D
:2041C000324801F06FFB80213048401C01F06AFB80212E48801C01F065FB80212B48C01C4B
:2041E00001F060FB80212948001D01F05BFB80212648401D01F056FB00212448801D01F034
:2042000051FB80210320800201F04CFB8021204801F048FB80211E48401C01F043FB802164
:204220001B48801C01F03EFB80211948C01C01F039FB00210D20000201F034FB80211548E4
:2042400001F030FB80211348401C01F02BFB80210720400201F026FB00210F48401F01F0EF
:2042600021FB80210C4801F01DFB80210A48401C01F018FB00BFCBE501020000010300005B
:2042800001040000010500000106000001070000010C0000060D0000060E000010B51448AF
:2042A0000078002808D013480078FF2804D01248FCF7A7FF0446A0470D484078002809D086
:2042C0000C484078FF2805D00B48A030FCF799FF0446A04706488078002808D0054880786C
:2042E000FF2804D00548FCF78CFF0446A04710BD00600040006100409D000020DD010020FE
:2043000010B50E480079002808D00D480079FF2804D00C48FCF775FF0446A047074840794C
:20432000002809D006484079FF2805D00548A030FCF767FF0446A04710BD00000060004065
:2043400000610040A200002010B50E48007A002808D00D48007AFF2804D00C48FCF751FF04
:204360000446A0470748407A002809D00648407AFF2805D00548A030FCF743FF0446A0477B
:2043800010BD00000060004000610040A700002010B50E48007B002808D00D48007BFF28BB
:2043A00004D00C48FCF72DFF0446A0470748407B002809D00648407BFF2805D00548A03058
:2043C000FCF71FFF0446A04710BD00000060004000610040AC00002010B50E48007C002802
:2043E00008D00D48007CFF2804D00C48FCF709FF0446A0470748407C002809D00648407C83
:20440000FF2805D00548A030FCF7FBFE0446A04710BD00000060004000610040B100002087
:2044200010B50E48007D002808D00D48007DFF2804D00C48FCF7E5FE0446A0470748407DB0
:20444000002809D00648407DFF2805D00548A030FCF7D7FE0446A04710BD000000600040D1
:2044600000610040B600002010B50E48007E002808D00D48007EFF2804D00C48FCF7C1FE58
:204480000446A0470748407E002809D00648407EFF2805D00548A030FCF7B3FE0446A047E3
:2044A00010BD00000060004000610040BB00002010B50E48007F002808D00D48007FFF287E
:2044C00004D00C48FCF79DFE0446A0470748407F002809D00648407FFF2805D00548A030C0
:2044E000FCF78FFE0446A04710BD00000060004000610040C000002010B50E480078002862
:2045000008D00D480078FF2804D00C48FCF779FE0446A04707484078002809D006484078FE
:20452000FF2805D00548A030FCF76BFE0446A04710BD00002060004020610040C5000020A2
:2045400010B50F480079002808D00E480079FF2804D00D48FCF755FE0446A0470848001DC3
:20456000407800280AD00748001D4078FF2805D00548A030FCF745FE0446A04710BD000010
:204580002060004020610040CA00002010B50E48007A002808D00D48007AFF2804D00C48FD
:2045A000FCF72FFE0446A047074808308078002809D0064808308078FF2804D00548FCF771
:2045C00020FE0446A04710BD2060004020610040CF0000200F02002010B50348FCF711FE0C
:2045E0000446A04710BD0000D400002010B50F48007C002808D00E48007CFF2804D00D480F
:20460000FCF7FFFD0446A04708481030407800280AD0074810304078FF2805D00548A030D0
:20462000FCF7EFFD0446A04710BD00002060004020610040D900002010B50348FCF7E1FD42
:204640000446A04710BD0000DE00002010B50348FCF7D7FD0446A04710BD0000E300002086
:2046600010B50F48007F002808D00E48007FFF2804D00D48FCF7C5FD0446A04708481C30F8
:20468000407800280AD007481C304078FF2805D00548A030FCF7B5FD0446A04710BD000051
:2046A0002060004020610040E800002010B514480078002808D013480078FF2804D01248B0
:2046C000FCF79FFD0446A0470D484078002809D00C484078FF2805D00B48A030FCF791FD60
:2046E0000446A04706488078002808D005488078FF2804D00548FCF784FD0446A04710BD44
:204700004060004040610040ED0000202D02002010B516480079002808D015480079FF28E3
:2047200004D01448FCF76DFD0446A0470F48001D407800280AD00E48001D4078FF2805D066
:204740000C48A030FCF75DFD0446A0470748001D8078002809D00648001D8078FF2804D0F4
:204760000548FCF74EFD0446A04710BD4060004040610040F20000203202002010B5164866
:20478000007A002808D01548007AFF2804D01448FCF737FD0446A0470F48083040780028AA
:2047A0000AD00E4808304078FF2805D00C48A030FCF727FD0446A0470748083080780028CA
:2047C00009D0064808308078FF2804D00548FCF718FD0446A04710BD406000404061004073
:2047E000F70000203702002010B51648007B002808D01548007BFF2804D01448FCF701FD8B
:204800000446A0470F480C30407800280AD00E480C304078FF2805D00C48A030FCF7F1FCD0
:204820000446A04707480C308078002809D006480C308078FF2804D00548FCF7E2FC0446DE
:20484000A04710BD4060004040610040FC0000203C02002010B51648007C002808D015486D
:20486000007CFF2804D01448FCF7CBFC0446A0470F481030407800280AD00E4810304078DB
:20488000FF2805D00C48A030FCF7BBFC0446A047074810308078002809D00648103080780F
:2048A000FF2804D00548FCF7ACFC0446A04710BD40600040406100400101002041020020D1
:2048C00010B50348FCF79DFC0446A04710BD00000601002010B50F48007E002808D00E4827
:2048E000007EFF2804D00D48FCF78BFC0446A04708481830407800280AD00748183040789E
:20490000FF2805D00548A030FCF77BFC0446A04710BD000040600040406100400B01002029
:2049200010B50F48007F002808D00E48007FFF2804D00D48FCF765FC0446A04708481C3096
:20494000407800280AD007481C304078FF2805D00548A030FCF755FC0446A04710BD0000EF
:2049600040600040406100401001002010B50E480078002808D00D480078FF2804D00C4896
:20498000FCF73FFC0446A04707484078002809D006484078FF2805D00548A030FCF731FC71
:2049A0000446A04710BD000060600040606100401501002010B50F480079002808D00E48D7
:2049C0000079FF2804D00D48FCF71BFC0446A0470848001D407800280AD00748001D407888
:2049E000FF2805D00548A030FCF70BFC0446A04710BD000060600040606100401A0100206A
:204A000010B51648007A002808D01548007AFF2804D01448FCF7F5FB0446A0470F48083028
:204A2000407800280AD00E4808304078FF2805D00C48A030FCF7E5FB0446A04707480830CB
:204A40008078002809D0064808308078FF2804D00548FCF7D6FB0446A04710BD60600040D5
:204A6000606100401F0100205F02002010B50348FCF7C7FB0446A04710BD0000240100206C
:204A800010B50348FCF7BDFB0446A04710BD00002901002010B51648007D002808D0154816
:204AA000007DFF2804D01448FCF7ABFB0446A0470F481430407800280AD00E4814304078B1
:204AC000FF2805D00C48A030FCF79BFB0446A047074814308078002809D0064814308078E6
:204AE000FF2804D00548FCF78CFB0446A04710BD60600040606100402E0100206E02002016
:204B000010B51648007E002808D01548007EFF2804D01448FCF775FB0446A0470F4818308F
:204B2000407800280AD00E4818304078FF2805D00C48A030FCF765FB0446A047074818302A
:204B40008078002809D0064818308078FF2804D00548FCF756FB0446A04710BD6060004044
:204B600060610040330100207302002010B51648007F002808D01548007FFF2804D0144876
:204B8000FCF73FFB0446A0470F481C30407800280AD00E481C304078FF2805D00C48A030E0
:204BA000FCF72FFB0446A04707481C308078002809D006481C308078FF2804D00548FCF746
:204BC00020FB0446A04710BD60600040606100403801002078020020F8B505460E4600205C
:204BE0000090ECB2602C01DB0120F8BDA00020181B49085C002801D00120F6E7A0002018DA
:204C0000174A8018411C3046FCF705FB0120A1006118134A505400222846EB17DB0E1B18EB
:204C20005B115B01EB1A9B000E4FDB19EF17FF0E7F197F11DA5503F0C3FD00222046E3171C
:204C4000DB0E1B185B115B01E31A9F00064BFB18E717FF0E3F197F11DA550098C5E700000A
:204C60009C00002000600040006100400A20704703208003FDF7B8FD401C002803D10D485A
:204C800003F076FD14E0FDF753FD0B4A51681068FDF7B8FB002808D103F06AFD0322920334
:204CA0001021064803F0A9FF02E0024803F060FD02F088FAA55AA55ABC3100200018500077
:204CC00000BFFEE710B572B631218902086880F3088800BF4868804710BD70B505460E462C
:204CE000002E05D031462846FCF730FA044600E02C46204670BD000070B505460E46FFF7C6
:204D0000B5FF04461D222146641C2048425400222146641C425409222146641C4254042204
:204D20002146641C4254290E2246641C81542802020E2146641C154842542804020E21464B
:204D4000641C124842542146641C4554300E2146621C94B20D4A50543002020E2046611CDA
:204D60008CB20A490A543004020E2046611C8CB206490A542046611C8CB204490E54044816
:204D80000178204601F046FC70BD0000D4310020DD02002070B50546FFF768FF04461D225A
:204DA0002146641C1048425400222146641C425401222146641C4254022D06D1022220464F
:204DC000611C8CB208490A5407E0032D05D103222046611C8CB204490A5404480178204660
:204DE00001F018FC70BD0000D4310020DD02002070B505460E46FFF739FF04461D2221467B
:204E0000641C1948425400222146641C425407222146641C425401222146641C4254290EFF
:204E20002246641C81542802020E2146641C0E4842542804020E2146641C0B484254214635
:204E4000641C45543004020E2046611C8CB206490A542046611C8CB203490E540348017894
:204E6000204601F0D7FB70BDD4310020DD02002010B50F480088002819D00D4840880028BE
:204E800015D0FFF7F3FE044601222146641C094842541C222146641C42540146081904499B
:204EA000FCF77EF91C340121204601F0B3FB10BDE0410020D4310020F8B507460D46164635
:204EC000FFF7D4FE044618222146641C12484254E81CC2B22146641C0F4842543002020E21
:204EE0002146641C0C4842543004020E2146641C094842542146641C4654014608192A4676
:204F00003946FCF74DF9601984B204480178204601F080FBF8BD0000D4310020DD020020BA
:204F200070B505460E46FFF7A1FE044619222146641C1A48425408222146641C4254310ECE
:204F40002246641C81543002020E2146641C134842543004020E2146641C104842542146FA
:204F6000641C4654290E2246641C81542802020E2146641C094842542804020E2046611CFC
:204F80008CB206490A542046611C8CB203490D5403480178204601F03DFB70BDD4310020B3
:204FA000DD020020F8B505460F461646FFF75EFE04461E222146641C19484254701D0004FE
:204FC000020E2146641C16484254701DC2B22146641C1348425401222146641C4254290E36
:204FE0002246641C81542802020E2146641C0C4842542804020E2146641C09484254214678
:20500000641C45540146081932463946FCF7C8F8A01984B203480178204601F0FBFAF8BDB1
:20502000D4310020DD020020F8B504460F4615461E4600200090002C1CD10120800285420E
:2050400015D8414806604148056001683E480068FCF7BFF8A9B23846FFF7CAFE01203C4948
:20506000087000203B4908603B4908606AE00120009067E0052C14D10120800285420DD819
:20508000AAB231463846FFF78DFF0120304908700020304908603049086053E00120009065
:2050A00050E0042C0CD129463846FFF725FE0120274908700020274908602749086041E0B3
:2050C000012C30D122480078012802D10220009038E01F480078022806D11E4800681E49E5
:2050E0000968401800902DE019480078032803D118480068009025E015480078052803D13F
:205100001648006800901DE011480078042806D110480068104909684018009012E00020E4
:205120000B4908700EE0022C01D0032C0AD12046FFF730FE01200649087000200549086064
:20514000054908600098F8BD3C000020400000203800002044000020480000204C00002000
:20516000FFB587B005460E461F46002479E33019791E0840285C022809D1601C3018084004
:20518000285C069000F0E8FDFFF772FE65E33019791E0840285C03287ED1601C3018084040
:2051A000285C0690A01C30180840285CFE490870E01C3018791E0840285CFB494870201D66
:2051C0003018791E0840285CF7498870601D3018791E0840285C0007C00FF4490870601DBC
:2051E0003018791E0840285C4007C00FF0490870601D3018791E0840285C0011ED49087056
:20520000601D3018791E0840285C8007C00FEA490870601D3018791E0840285CC007C00FA7
:20522000E6490870A01D3018791E0840285C0002E11D71187A1E1140695C0843E04908802C
:20524000204608303018791E0840285C00022146093171181140695C0843D9494880204628
:205260000A303018791E0840285C000221460B3171181140695C0843D149888020460C30F6
:205280003018791E0840285C000221460D3171181140695C084300E016E0C949C88020463C
:2052A0000E303018791E0840285CC007C00FC549087020460E303018791E0840285C800713
:2052C000C00FC1490870C8E23019791E0840285C052819D1601C30180840285C0690BB48E7
:2052E00000680028EFD000200AE0A11C091889197A1E1140695CB54A12681154411CC8B272
:2053000006998842F1DBA8E23019791E0840285C152820D1601C30180840285C0690A01C12
:2053200030180840285CAA490870E01C3018791E0840285CA6494870201D3018791E08403C
:20534000285CA3498870601D3018791E0840285C9F49C87081E23019791E0840285CC8289E
:2053600014D1601C30180840285C0690E01C30180840285C974909788842A4D1201D3018ED
:20538000791E0840285C9349487066E23019791E0840285C182854D1601C30180840285C2D
:2053A0000690A01C30180840285C0590059800020590E01C30180840285C05990843059030
:2053C000059800020590201D3018791E0840285C059908430590059800020590601D30183A
:2053E000791E0840285C059908430590A01D3018791E0840285C0490049800020490E01DA1
:2054000030180840285C0499084304907248006800289FD07148006800289BD004980028CB
:2054200098D00499059840186C490968884291D869490A68059950180A460499FFF73CFDD3
:205440000BE23019791E0840285C19280BD1601C30180840285C069060480168604800684F
:20546000FFF75EFDF9E13019791E0840285C1B280BD1601C30180840285C0690E01C3018CC
:205480000840285C57490870E7E13019791E0840285C1D287ED1601C30180840285C00028E
:2054A000A11C71187A1E1140695C08430690E01C3018791E0840285C01284AD102A903A8D6
:2054C000FEF734FC0398002842D00698401F029988423DD800200AE02146083109188919EE
:2054E0007A1E1140695C039A1154411C88B20699491F8142F0DC201D3018791E0840285CE7
:205500000390039800020390601D30180840285C039908430390039800020390A01D301888
:20552000791E0840285C039908430390039800020390E01D3018791E0840285C03990843CF
:2055400003900698421F00231846039900F03AFE10E1E01C3018791E0840285C02287DD164
:20556000201D30180840285C0390039800020390601D30180840285C039908430390039871
:2055800000020390A01D3018791E0840285C0399084300E0F3E00390039800020390E01DB4
:2055A0003018791E08401FE0F0020020DD020020DF020020DE020020E0020020E1020020AE
:2055C000F4020020E2020020E3020020D8020020D4020020D4410020E4020020E802002077
:2055E000EC020020DC020020285C039908430390204608303018791E0840285C029002982C
:20560000000202902046093030180840285C02990843029002980002029020460A303018B5
:20562000791E0840285C02990843029002980002029020460B303018791E0840285C02997A
:205640000843029020460C303018791E0840285C0190019800020190204600E025E00D30DB
:2056600030180840285C01990843019001980002019020460E303018791E0840285C01998B
:205680000843019001980002019020460F303018791E0840285C0199084301900120019B7F
:2056A000029A039900F08EFD64E0E01C3018791E0840285C03282BD1201D30180840285CD4
:2056C0000390039800020390601D30180840285C039908430390039800020390A01D3018C7
:2056E000791E0840285C039908430390039800020390E01D3018791E0840285C039908430E
:20570000039000231A460120039900F05BFD31E0E01C3018791E0840285C04282AD1201D52
:2057200030180840285C0190019800020190601D30180840285C01990843019001980002F6
:205740000190A01D3018791E0840285C019908430190019800020190E01D3018791E08408A
:20576000285C019908430190002211460320019B00F028FD0698401C80B206906DE030198A
:20578000791E0840285C1E2866D1601C30180840285C0002A11C71187A1E1140695C084358
:2057A0000690201D3018791E0840285C0390039800020390601D30180840285C0399084330
:2057C0000390039800020390A01D3018791E0840285C039908430390039800020390E01DF7
:2057E0003018791E0840285C039908430390204608303018791E0840285C0290029800020D
:2058000002902046093030180840285C02990843029002980002029020460A303018791E1E
:205820000840285C02990843029002980002029020460B303018791E0840285C02990843C4
:20584000029000220220029B039900F0BBFC0698401C80B2069000E007E00698801C201897
:2058600084B20998844200DA81E400BF0BB0F0BD10B501231A4600211846FCF71DFB01222F
:2058800011461046FCF784FBFBF71CFC034803F073F802480249086010BD00000090D00309
:2058A000C4020020FEB505460C460020C0430290EFB22804060E0F2E42DA082F40DA012051
:2058C000B8406946088080202040002816D101208870A007800F022801D1487109E0A007F6
:2058E000800F012802D16946487102E0002069464871F0B26946FDF76BFF1FE000206946CE
:2059000088700E202040002800D000BF10202040002802D16946087102E00120694608716C
:20592000E007C00F002802D16946887102E0012069468871F0B26946FDF74AFF0020029023
:205940000298FEBD01220B490A710A720A730A740A750A764A714A724A734A744A754A7619
:20596000002004E000218200034B9950401C0C28F8D3704700610040141A0020F8B5044651
:205980000F460020C0430090E6B22004050E0F2D11DA082E0FDA0120B04086B2002F04D19D
:2059A000E8B23146FEF70EF803E0E8B23146FEF70FF8002000900098F8BD000010B50548DC
:2059C0000068002802D003480068804700F04EFC10BD00008400002070B504460D46601E00
:2059E0000D49884200D90124002C00D1012440200A490870084600786043094948610321B4
:205A0000081F02F0E9FE002005498861072008610448056070BD0000FFFFFF00880000201C
:205A200000E000E0840000200020C043002809DBC206D20E01219140054A1160BFF34F8FE8
:205A4000BFF36F8F00BF0020024908618861704780E100E000E000E0F0B587B006460C46E8
:205A6000002700216846C1820020039068468182418201824183018300F002F9032E7DDA88
:205A8000206800287AD060680028FBD0002E04D0012E3ED0022E72D17CE0674D00231F222B
:205AA00002210520FDF738FF00231E2201210520FDF732FF0221684681800021817101724C
:205AC000012181720021C17101A90520FDF780FE01216846818081710021C17101A9052038
:205AE000FDF776FE6068039007216846018210214182002181824183802101833221C182F3
:205B00004E490A20FFF768F84D490B20FFF764F881E0494DAD1C0023032204211846FDF7DC
:205B2000FBFE0023042208211846FDF7F5FE04216846818000218171017201218172002125
:205B4000C17101A90020FDF743FE082168468180012181710021C17101A90020FDF738FEE1
:205B6000606803900721684601821021418200218182418380210183322101E058E049E0DB
:205B8000C18230490D20FFF727F82F490E20FFF723F840E02D4D10232E2240210720FDF7B7
:205BA000BBFE11232F2280210720FDF7B5FE8021684681800021817101720121817200212C
:205BC000C17101A90720FDF703FE402168468180012181710021C17101A90720FDF7F8FD9C
:205BE0006068039007216846018210214182002181824183802101833221C1821449E068B5
:205C0000C86014490720FEF7E7FF13490820FEF7E3FF00E000BF00BF03A9284601F010F930
:205C20000746002F04D0CD220CA1384602F07EFF606807B0F0BD0000101000000D6C0000C6
:205C4000B96B0000B56C0000616C000010200000041A00205D6D0000096D00002E2E5C5379
:205C60006F757263655C436F6D706F6E656E745C554152545C5254455F554152542E6300EC
:205C800000200F49086048600872C8600D49086048608860C8600C49086048600872C8605D
:205CA0000A49086048608860C8600949086048600872C8600749086048608860C860704746
:205CC000B4190020E4190020C4190020F4190020D4190020041A002010B502F02DFC10BD98
:205CE0001A20084908722B2048723C2088724D20C8727F20044909680860AC200349487008
:205D000070470000000402408C0000200010024010B504460F488088002800D110BD0D48FF
:205D20000088182250430B4A0832811818222046FBF736FA07490988481C1721FBF71CFA9F
:205D400088B20449088008468088401E88800120E4E70000841700200020054908600549AD
:205D600008600549087005490870054908707047CC020020D0020020DD020020DE020020D3
:205D8000E002002000B519480078012813D118480078012804D100201549087015490870C4
:205DA00014480078322801DB01F00CFA11480078401C1049087010480078012814D10F48AF
:205DC000007864280BD300200B4908700C480078801E0B49087000200849087004E00748A3
:205DE0000078401C0549087000BD00009402002096020020950200209A0200209B020020AE
:205E0000A8020020F8B504460D460026002700200090201300F09AF900901448844205D034
:205E2000801C844202D01248844217D122202840222806D127073F0F39460098FBF71CFCBE
:205E400006461220284012280ED12007000F471C39460098FBF710FC064605E02107090F24
:205E60000098FBF709FC06463046F8BD1010000010200000FFB58BB01C460020079006902E
:205E800005903848049010210B980840002801D0022707E040210B980840002801D00127C7
:205EA00000E00027002C04D0149804700120089001E010200890002548E0002C08D025469D
:205EC0006000294A115A0C98FBF740F9079006E06800254A115A0C98FBF738F907903E4614
:205EE00030E0711C0798FBF731F9400806900D98FBF715FA03900D9A0699881AFBF70FFA50
:205F000018490190FBF790F902900399FBF7C9F905900598FBF70AFA49004908039102904A
:205F20000498FBF703FA4900490801910090039B029AFBF70FFA03D20A95099605980490A1
:205F4000701CC6B27F2ECCDD681CC5B208988542B3DB14990A98087014990998487004988E
:205F60000FB0F0BD0000C842DE8E000010B50246374BD01A9A4233D014DC364BD01A9A42B0
:205F80002DD008DC34481018002846D002284CD010285AD11DE0012827D002282BD01F280C
:205FA00053D117E02B4C423C031BA04229D009DC01281BD002281FD0274B4133C0180028E0
:205FC00043D13AE0012B22D0202B1BD0212B3CD11EE000BF214803890B43038136E000BF8D
:205FE0001E4843890B43438130E000BF1B4883890B4383812AE000BF1848C3890B43C381C6
:2060000024E000BF164883880B4383801EE000BF1348C3880B43C38018E0104843890B43A5
:20602000438103890B43038110E00C48C3890B43C38183890B43838108E00948C3880B43EC
:20604000C38083880B43838000E000BF00BF10BD4110000021100000F0EFFFFF00110440C2
:206060000014044030B502460020334C131BA24233D014DC314C131BA2422DD008DC304B0C
:20608000D318002B46D0022B49D0102B51D11DE0012B27D0022B2BD01F2B4AD117E0274D19
:2060A000423D5C1BAB4229D009DC012B1BD0022B1FD0234C41341B19002B3AD134E0012C5D
:2060C00022D0202C1BD0212C33D11EE000BF1D4B1C880C40E0B22DE000BF1A4B5C880C403E
:2060E000E0B227E000BF174B9C880C40E0B221E000BF144BDC880C40E0B21BE000BF124B6C
:206100001C880C40E0B215E000BF0F4B5C880C40E0B20FE00B4B5C880C40E0B20AE0094BE8
:20612000DC880C40E0B205E0074B5C880C40E0B200E000BF00BF30BD411000002110000057
:20614000F0EFFFFF001104400014044030B50246002100230024002000BF0BE001258D4063
:20616000EBB215461D402C469C4201D1084603E04D1CE9B20429F1D300BF30BD00BF0948C6
:206180000068094948430949401806490860084600680028F3D008460068401C0028EED0C0
:2061A00070470000A00200206D4EC6413930000010B504461C2221460148FAF7F1FF10BD90
:2061C000E041002030B50F4C21600F4C22600F4C2360002803D102240D4D2C7010E00128D1
:2061E00003D103240A4D2C700AE0022803D10424074D2C7004E0032802D10524044D2C70B9
:2062000030BD000044000020480000204C000020380000200149086070470000D80200209E
:2062200010B504480068401E02490860FFF7C6FB10BD00009800002010B5FFF7A3FD10BD70
:2062400010B50A20FBF7D0FF10BD704710B57D200001FDF7AFF903480078012801D102F05B
:206260005DF910BDC00200207047704710B5FDF729FD0F480068401C0D490860084600683D
:20628000142806D3002008600A480068401C0949086009480088401C0749088008460088AE
:2062A000282804DB002008800220FBF7ADF910BD90020020880200208C0200200CB500BFF6
:2062C000054800680090044800680190019900988842F5D100980CBD8402002010B5FBF7B4
:2062E00073FAFCF7DAFA00F0CDFF10BD70B5314800683149096840182E4908600846006803
:206300007D21C900884211D32A480068FAF71EFF06467D21C90027480068FAF717FF254882
:20632000016026480068801924490860244840682149096840182249486008460068002880
:2063400037D10025084684682EE02068002829D01B49606849680022D243511A884205D2FF
:206360001749606849684018606002E00020C0436060A1686068884214D3206801280AD159
:2063800000202060002D03D10D492069886004E02069286101E000206060E068002801D09D
:2063A000E068804725462469002CCED100200449486070BD800200207C02002084020020E3
:2063C0006C1A002010B5FFF72FFB322000F008F802493220FFF700FB10BD0000ED62000046
:2063E00010B504460D48046000200D4908600D4908600D49086048608860FFF75FFF0B4943
:2064000008600020486088600120C86003200861052048610720886110BD00007C02002046
:2064200080020020840200206C1A0020501A002070B5FFF753FFFFF741FF05463A4800680C
:20644000A84203D8384800682C1A06E0364800680021C943081A4019441C334805604068ED
:2064600000193149486008464068022806D308460079C007C00F4860FFF7E8FE2A488068AD
:2064800000192949886008468068052807D388680521FAF75BFE24488160FFF7E6FE22485B
:2064A000C06800192049C8600846C0680A2807D3C8680A21FAF74AFE1B48C160FFF7C0FEBC
:2064C0001948006900191849086108460069142807D308691421FAF739FE13480161FFF7C1
:2064E000B4FE1148406900190F49486108464069322807D348693221FAF728FE0A48416194
:20650000FFF7B2FE0848806900190749886108468069642807D388696421FAF717FE0248E7
:206520008161FFF789FE70BD501A00201FB5FFF7D7FBFFF79DF9FFF745FF0E48FDF7BCFBE2
:20654000FFF700FA0020FDF75FFCFBF799FE0A48007801280DD10090E120400201900020FE
:2065600002900648039069460220FFF775FAFBF797F81FBDD95C0000C0020020991700004E
:2065800010B580201B4948711A201A49203908722B2048723C2088724D20C8720020164988
:2065A0004860FBF725FD154908600020C0431449086014490860144814490860114903220C
:2065C0001202891848600F49891888600D498918C8600C49891808610A4989184861094910
:2065E0008918886107498918C861AC200849487010BD00002004024000B00140C402002018
:2066000080E200E000E100E0C0C0C0C000E400E000100240F3B583B007463C460294049885
:20662000002845D00A2C3FDD0020C04322460A3A01231B030A2100901E48FBF783FD0646DB
:2066400025460024EB222146641C1A48425490222146641C42542804020E2146641C154810
:2066600042542146641C45542812C043C2B22146641C10484254E843C2B22146641C0D48A3
:206680004254310E2246641C81543002020E2146641C084842543004020E2146641C0548E1
:2066A00042542146641C46540248029901F02EFF05B0F0BDD4310020F8B503460C460021D0
:2066C000012000900025608922263040222826D10720014319812021A07A0007000F014348
:2066E000084628430146198204214803014320890143A0890143E0880143A088014319833D
:2067000021200001C05A7F267602B043567876027F277F023E40304321263601F052608906
:206720001226304012283BD100210720014359813F48007C012630433D4E307420210846AA
:206740002843014600BFB0150143E08901430220014300BF59820421400301432089014379
:20676000A089014310200143A088014359833148C05A7F267602B043567876027F277F02E0
:206780003E4030432B4EF052998EE089002804D10E4600988643314601E0009801439986B8
:2067A000608912263040122804D1988C80088000801C9884608922263040222804D1988C71
:2067C00080088000401C9884DE8C0020DE8C360936010643DE84D88C0009000116783607EB
:2067E000360F3043D88460891226304012280BD1588D0226B0435885188DB0431885588CE8
:2068000080088000801C588460892226304022280BD1188D012630431885588D3043588520
:20682000588C80088000401C58840020F8BD00006004044012020000F8B503460C4600213A
:20684000042000904503608922263040222826D10720014399812021A07A0007000F014320
:20686000084628430146998204214803014320890143A0890143E0880143A08801439983BB
:2068800085208000C05A7F267602B043567876027F277F023E4030438526B600F0526089BF
:2068A0001226304012283BD1002107200143D9815448007C04263043524E3074202108467C
:2068C0002843014600BFB0150143E08901430220014300BFD9820421400301432089014378
:2068E000A089014310200143A0880143D9834648C05A7F267602B043567876027F277F02CA
:206900003E403043404EF052998EE089002804D10E4600988643314601E000980143998621
:20692000608912263040122804D1988C0C26B04308309884608922263040222804D1988C36
:206940000C26B043001D9884DE8C3606360F00263601F0273E403046DE8CBE430643DE8470
:20696000D88CF026B043167836013E403043D88460891226304012281ED15E8D3607B60FF1
:206980000227BE43B6000C273E4030465E8DBE4306435E851E8D3607B60F0227BE43B6004B
:2069A0000C273E4030461E8DBE4306431E85588C0C26B04308305884608922263040222810
:2069C0001ED11E8D3607B60F01273E43B6000C273E4030461E8DBE4306431E855E8D3607D5
:2069E000B60F01273E43B6000C273E4030465E8DBE4306435E85588C0C26B043001D588432
:206A00000020F8BD6004044016020000F8B503460C46002101200090002560892226304001
:206A2000222825D10720014399802021A07A0007000F0143084628430146198104214803D3
:206A4000014320890143A0890143E0880143A08801439981F000C05A7F267602B04356787E
:206A600076027F277F023E403043FF261136F05260891226304012283DD100210720014373
:206A8000D9804C48007C102630434A4E3074202108462843014600BFB0150143E0890143F2
:206AA0000220014300BF598104214003014320890143A089014310200143A0880143D98197
:206AC000FF201330C05A7F267602B043567876027F277F023E403043FF261336F052198C77
:206AE000E089002804D10E4600988643314601E0009801431984608912263040122804D10A
:206B0000988A80088000801C9882608922263040222804D1988A80088000401C9882DE8ACD
:206B20000020DE8A360936010643DE82D88A0009000116783607360F3043D8826089122644
:206B40003040122817D15E8B0227BE43B007800F5E8BB608B60006435E831E8BBE43B00762
:206B6000800F1E8BB608B60006431E83588A80088000801C5882608922263040222817D14C
:206B80001E8B01273E43B007800F1E8BB608B60006431E835E8B3E43B007800F5E8BB608FF
:206BA000B60006435E83588A80088000401C58820020F8BD600404401CB500200F49087394
:206BC00007210F4800F028F9009069460878002807D007210A4800F017F96846007801F0D6
:206BE000A8FF0848807C01900748C068002804D00548C1686846007988471CBD2060004099
:206C00001010000000130440E419002010B500200F4908720F4800680E49496888420BD2BB
:206C20000C4801680068401C0A4A10601046C068405C0949087409E0002006490872074806
:206C40008068002802D005498868804710BD000020600040B419002000130440E41900205F
:206C60001CB500200F49087607210F4800F0D4F8009069460878002807D007210A4800F0EA
:206C8000C3F86846007801F054FF0848807D01900748C068002804D00548C16868460079E1
:206CA00088471CBD206000401210000000130440F419002010B500200F4908750F4800684D
:206CC0000E49496888420BD20C4801680068401C0A4A10601046C068405C0949087509E0EE
:206CE00000200649087207488068002802D005498868804710BD000020600040C4190020EB
:206D000000130440F41900201CB500200F49087007210F4800F080F8009069460878002860
:206D200007D06846007801F004FF0721084800F06BF80848807C01900748C068002804D047
:206D40000548C1686846007988471CBD206000401020000000150440041A002010B5002082
:206D60000F4908770F4800680E49496888420BD20C4801680068401C0A4A10601046C0680B
:206D8000405C0949087409E000200649087207488068002802D005498868804710BD0000B4
:206DA00000600040D419002000150440041A002000200649098860221140002903D1044972
:206DC000097A002900D001207047000000140440D419002010B503460C46FFF7E9FF002894
:206DE0000CD101200649086008464460012008720846C360C06800780249087410BD0000AC
:206E0000D41900200015044070B504460D4629462046FFF7ABF870BD70B505460E46314674
:206E20002846FFF71FF9002801D0012400E00024204670BD0148006870470000C4020020D3
:206E4000F0B585B004460D460020039069892046FEF7D8FF40B203900398002802D003982F
:206E600005B0F0BD55482018002809D002282DD001210903401A4FD04900401A72D172E0D4
:206E8000A0120121FBF764F84D4FFFF7D3FF019002A80090F88C03071B0F2A682046019957
:206EA000FEF7E8FF06463046FAF740FA0022454B01910090FAF74EFA02D20520C043CFE74A
:206EC00002AA29463846FFF7F7FB73E0A0120121FBF73EF83A4FFFF7ADFF019002A80090EC
:206EE000F88C0006030F2A6820460199FEF7C2FF06463046FAF71AFA0022324B0191009026
:206F0000FAF728FA02D20520C043A9E702AA29463846FFF791FC4DE0A0120121FBF718F8B3
:206F2000294FFFF787FF019002A80090F88A03071B0F2A6820460199FEF79CFF06463046F8
:206F4000FAF7F4F900221F4B01910090FAF702FA02D20520C04383E702AA29463846FFF7C3
:206F600055FD27E025E0E0120121FBF701F8174FFFF760FF019002A80090F88A03071B0F78
:206F80002A6820460199FEF775FF06463046FAF7CDF900220B4B01910090FAF7DBF902D24A
:206FA0000520C0435CE702AA29463846FFF72EFD00E000BF00BF039852E70000F0EFFFFF9D
:206FC000001104400000F03F00140440001604401FB504460A4800900021684641710821D1
:206FE0008171032101727F21417284727821C172AA21017341738173C173FBF7D3F91FBD3E
:207000008907000000B503460A46002A03D1184600F010F903E00121184600F00BF900BD29
:207020007047F0B505460E4617461C46002C05D13A463146284600F0FFF805E001233A46BF
:207040003146284600F0F8F8F0BD70B504460D461646324629462046FBF7B2FE70BD000084
:2070600010B50020044908700449087004490860FCF796FB10BD00009C0200209D0200201E
:20708000A40200201CB5002001904848007A00287ED00020464908704648007931282DD0A4
:2070A00008DC10280FD011284CD0222814D027285AD11AE034282AD0362831D0372838D0C2
:2070C0003E2851D147E0394A203AD18C394A1068521D00F0DBF859E0344A203AD18C354AAD
:2070E0001068521D00F01CFA50E0304A203AD18C304A1068521D00F009FB47E02B4A203AF7
:20710000D18C2C4A1068521D00F028FC3EE0274A203AD18C274A1068521D00F059FE35E0A7
:20712000224A203AD18C234A1068521D00F048FF2CE01E4A203AD18C1E4A1068521D01F036
:2071400081F823E0194A203AD18C1A4A1068521D00F054F91AE0154A203AD18C154A10682A
:20716000521D01F0CDF811E012480068124988420BD01120019001A80E4900900879012340
:207180000D4A563A194601F039F900BF00BF00E00BE000200549087208480078012804DD83
:2071A000012007490870024908701CBDE42700209402002004230020DF0700009702002083
:2071C0009602002000BFBFF34F8F04480449C860BFF34F8F00BF00BF00BFFDE70400FA0533
:2071E00000ED00E01FB51048007801281BD10F4800900021684641710821817106210172EC
:2072000050214172022181720021C1723221017301214173F4218173AA21C173FBF7C2F88F
:207220000120034908701FBD99020020890700009402002070470000F0B50446002B12D1D8
:207240000125094E3572094D2C60551E203EF584002006E00E78054D2D1D2E54491C451C6E
:20726000A8B29042F6DBF0BDE42700200423002070B504460D461646324629462046FFF791
:20728000E4FE70BD10B5FFF7FDFE10BDF7B584B00E46102003900024374604980290002076
:2072A0000190002F03D113204F49087002E000204D4908704C48007800281AD1002505E0BE
:2072C0000698405D49494855681CC5B2BD42F7DB4648007880210840C0090190434800782C
:2072E0004406640E002C01D0032C02D912203E4908703D480078002804D1012F02D013206B
:207300003949087038480078002812D1022C07D13748007801280CD17E203349087008E0F3
:20732000032C06D132480078022802D17E202E4908702D48007800282AD12C49487032203C
:2073400088700120C870F4200871012C10D10198002807D108460523264A00210090039876
:2073600001F04CF832212448FCF7B4FCFFF72AFFFFF776FE1E4804700198002832D11B48EC
:2073800005231C4A00210090039801F037F829E018495631029888421CD1134800781128A5
:2073A00020D01148007812281CD00F4800787E2818D00D4800787F2814D00B48007831280D
:2073C00010D0094801230B4A19460090039801F015F807E004480123064A1946009003984A
:2073E00001F00CF807B0F0BD98020020C0280020970200208907000050C30000F7B586B034
:2074000006460F4611200590002004903D46039602903E480078012803D17F203C4908700C
:2074200002E000203A49087039480078002804D1012D02DA13203649087035480078002808
:207440001AD1002405E00898005D32490855601CC4B2AC42F7DB2F48007880210840C00910
:2074600002902C4800784006400E04900498012802D012202649087025480078002804D1D4
:20748000012D02D013202249087021480078002810D10298002837D11E4801231E4A00210F
:2074A0000090059800F0AAFF32211C48FCF712FCFFF788FE18495631039888421CD114483C
:2074C0000078112820D01248007812281CD0104800787E2818D00E4800787F2814D00C4808
:2074E0000078312810D00A4801230B4A19460090059800F083FF07E005480123064A19460B
:207500000090059800F07AFF09B0F0BD9702002098020020C02800208907000050C3000051
:20752000F7B584B00E4622200390374604980290022F03DA13206949087002E0002067497A
:20754000087066480078002822D1002505E00698405D63494855681CC5B2BD42F7DB604870
:20756000007804025E4949780C435E4884420FD05C480E3084420BD0801E844208D0801D2F
:20758000844205D05848844202D031205349087052480078002804D1022F02D013204F49D6
:2075A00008704E48007800286BD14E490C31601A8C422CD008DC4D482018002845D04C4946
:2075C0004018002850D104E0022811D006284BD12CE00F2247494248801CF9F7E1FD404888
:2075E0001123454A00210090039800F007FF47E0092242493A48801CF9F7D2FD38480B231E
:207600003D4A00210090039800F0F8FE38E009223B493348801CF9F7C3FD31480B23364AFC
:2076200000210090039800F0E9FE29E0042235492B48801CF9F7B4FD294806232E4A002197
:207640000090039800F0DAFE1AE00D222E492448801CF9F7A5FD22480F23274A002100903F
:20766000039800F0CBFE0BE031201C49087008460123214A19460090039800F0BFFE00BFCA
:2076800029E01D495631029888421CD113480078112820D01148007812281CD00F480078E1
:2076A0007E2818D00D4800787F2814D00B480078312810D0094801230F4A19460090039888
:2076C00000F09CFE07E0054801230B4A19460090039800F093FE07B0F0BD0000980200204A
:2076E000C028002087F1000024100000DCEFFFFF9D1EFFFF90930000890700009F9300006F
:20770000A8930000B1930000B5930000F7B584B0272002900024059E04980190854901988E
:20772000884203D111208449087002E000208249087081480078002806D180480078022846
:2077400002D07F207C4908707B480078002804D1002E02D113207849087077480078002877
:2077600012D1002505E00698405D75494855681C85B2B542F7DB72480478112C04D0122C7D
:2077800002D012206C4908706B48007800280CD1112C05D1012E08D013206749087004E02F
:2077A000052E02D013206449087063480078002808D1122C06D163480078012802D02420D1
:2077C0005D4908705C480078002808D1112C06D15D480078012802D1372057490870564834
:2077E0000078002879D1112C02D0122C76D142E056480078022808D111205149087000206D
:2078000048708870C870087116E0FEF7B7FC50480068000E4A4948704D4800680002000E03
:2078200088704B4800880004000EC870484800780871012043490870414805233D4A563A7D
:2078400000210090029800F0D9FD3D484178684601733B488178684641733948C178684671
:207860008173374801796846C17303A8FAF78EFC384908604DE00020324908703048401C16
:20788000FAF7F0FE07463348006887420CD102202E4908702A480123264A563A00210090DB
:2078A000029800F0ABFD26E02B480078401C2A49087008460078032811DB0120224908707D
:2078C00036201D490870084601231A4A563A19460090029800F092FD0DE01BE00CE03520DD
:2078E0001549087008460123124A563A19460090029800F083FD0CE012200F49087008461F
:2079000001230C4A563A19460090029800F076FD00BF0DE007495E390198884208D1064854
:207920000123044A563A19460090029800F066FD07B0F0BDDF0700009802002097020020AC
:20794000C02800209C0200209A0200209D020020A0020020A4020020A8020020F7B58AB0AE
:2079600031200490002003900B9D0A9802900026F7490298884203D11120F649087002E02B
:207980000020F4490870F3480078002806D1F2480078022802D07F20EE490870ED480078B7
:2079A000002806D1ED480078022802D03320E9490870E8480078002804D1032D02D2132046
:2079C000E4490870E3480078002812D1002405E00C98005DE2490855601C84B2AC42F7DB50
:2079E000DF48007803900398012802D01220D9490870D848007800282BD1D948407800025C
:207A0000D749897808430646FF200002864217D1D348001DFAF726FE0990D1480830FAF7B5
:207A200021FE0890032189030998884204D11D218903089888420CD93120C649087008E0C6
:207A4000C848864205D0C848864202D03120C1490870C0480078002822D1F01FFF38FC38E7
:207A600000280CD0C1494018002802D0012812D10BE00C2D02D01320B64908700FE0072DD7
:207A800002D01320B349087009E0032D02D01320B049087003E03120AE49087000BF00BFBD
:207AA000AC48007800287DD1F01FFF38FC38002806D0AE494018002875D0012874D11DE144
:207AC000A748C0780006A649097909040843A449497909020843A249897908430590A448F2
:207AE000007D002840D1A3480068C043A149086005980968884227D19F4800783E2813D1AF
:207B00000020C0439B49086001209949087500209349C870084604238D4A563A00210090B5
:207B2000049800F06BFC60E000219148017501208B49C87008460423854A563A00210090F0
:207B4000049800F05BFC50E000208949087501208349C870084604237D4A563A0021009001
:207B6000049800F04BFC40E08448008A8349498A884206DB8148008A8049498A401A80B2F7
:207B800006900698002806D07C494A8A14315018069900F06DFE77480068C0437549086023
:207BA000059802E001E121E0F2E0096888420CD100206B49C87008460423654A563A002198
:207BC0000090049800F01AFC0BE001206449C870084604235E4A563A00210090049800F098
:207BE0000DFC0020C04363490860DDE06048007D012873D10498FFF7EBF90020604908703F
:207C0000FAF7C4FDFAF794FD002007905D4880680121C904884205D25A4800686121490285
:207C2000884212D05848806823214903884205D25548006861214902884202D001200790B9
:207C40001FE0FAF735FD07901BE04E4A51681068FAF7D8FB002811D103208003FAF7C4FD81
:207C6000074623204003FAF7BFFD874202D10120079006E0FAF71CFD079002E0FAF718FDC1
:207C800007900798012818D1404800F071FD232149030320800300F07DFE012034494875BA
:207CA00000202F49C87008460423294A563A00210090049800F0A2FB1FE000202C49487551
:207CC00072202449087008460123214A563A19460090049800F092FB0FE0FFE70021244856
:207CE000417501201E49C87008460423184A563A00210090049800F081FB55E01F4A916857
:207D00005068FAF77FFB002812D10498FFF760F9002000F02DFD00201149C87008460423E9
:207D20000B4A563A00210090049800F067FB0EE000210F48017501200949C87008460423C3
:207D4000034A563A00210090049800F057FB2BE0DF07000098020020970200209D02002094
:207D6000C02800200202000001FF00000203FFFFA4310020AC020020A9020020A42D002075
:207D8000C0020020C8310020BC310020A55AA55A31200D490870084601230C4A1946009007
:207DA000049800F02BFB00BF0CE0084908390298884207D104480123044A1946009004984F
:207DC00000F01CFB0DB0F0BD9802002089070000F7B586B0064600250027342005900798E6
:207DE000049003966C4802906C48039E864203D111206B49087002E00020694908706848E6
:207E00000078002806D167480078022802D07F206349087062480078002806D162480078C2
:207E2000022802D033205E4908705D480078002805D104980A2802D013205949087058482C
:207E40000078002815D1002405E00898005D57490855601C84B204988442F6DB53480078A1
:207E6000002803D151484078442802D031204C4908704B48007800287ED14D4908704B48F6
:207E8000801CFAF7EFFB05464848801DFAF7EAFB07464848007D012847D14648407D01280E
:207EA00036D103208003854225D11D208003874221D241480560E81DFF30FA303E49486061
:207EC000F81FFF38FA388860202038490870042048700220887008460323304A563A00216C
:207EE0000090059800F08AFA01203249887500203149C8604EE031202949087008460123AB
:207F0000264A563A19460090059800F077FA41E070202349087008460123204A563A194614
:207F20000090059800F06AFA34E02448854216D1202F14D101201F49887520201B490870BC
:207F4000042048700220887008460323134A563A00210090059800F051FA1BE00CE0312009
:207F60000F490870084601230C4A563A19460090059800F043FA0DE008495E3903988842E6
:207F800008D107480123054A563A19460090059800F034FA09B0F0BD02040000DF070000BA
:207FA00098020020970200209D020020C0280020A9020020A4310020A42D002000009F0136
:207FC000F7B5FFB0FFB088B006460021FFA88161416136210391056A02969148029E864294
:207FE00003D111208F49087002E000208D4908708C480078002806D18B480078022802D04A
:208000007F208849087087480078002806D187480078022802D03320824908708148007818
:2080200000280FD1681E8249C8600846C068002805D00846C06801218902884202D9132051
:20804000784908707748007800281ED1002406E0FFA8406A005D77490855601C84B2AC4224
:20806000F6DB744800787449897D88420AD17248807DFFA988617048807D401CC1B26E4811
:20808000817502E073206749087066480078002875D16948007D012872D1654800680321E6
:2080A000890388425BD3624800680121C904884255D200244EE0FFA8406A001941785C4831
:2080C000028A143081541438008A401C5849088208460068594988423AD25548008A012127
:2080E0008902884234D3FF2204A8F9F76BF800270CE04F48418A1430405C04A9C8554C4851
:20810000408A401C4A494882781C87B2012080028742EED301464648143000F0A9FB4449A8
:2081200004AA08680121890200F067FD0146FFA84161406900280AD13D480068012189024A
:2081400040183B49086000200882488200E005E0601C84B23648C068A042ACD811E0722061
:2081600030490870084601232D4A563A19460090039800F043F97FB07FB00BB0F0BD3FE0FA
:208180001EE0FFA8406900280DD1FFA880692949087008460123224A563A00210090039857
:2081A00000F02CF93AE072201E490870084601231B4A563A19460090039800F01FF9DAE765
:2081C000012408E01B48005D1D49097840181C490870601C84B2AC42F4DB691E1548401C07
:2081E00000F046FBFFA8806912490870084601230B4A563A00210090039800F0FFF80DE074
:2082000007495E390298884208D106480123044A563A19460090039800F0F0F800BFAAE738
:20822000DF07000098020020970200209D020020A42D0020C0280020A431002000FC070035
:20824000A9020020FEB504460D46372001902F4626462548864203D111202449087002E039
:2082600000202249087021480078002806D120480078022802D07F201C4908701B480078E8
:20828000002806D11B480078022802D033201749087016480078002804D1002F02D01320D6
:2082A000124908701148007800280ED1FAF72AF9002011498875114800230B4A563A1946C8
:2082C0000090019800F09AF80CE007485E38864208D106480123044A563A194600900198A9
:2082E00000F08CF8FEBD0000DF07000098020020970200209D020020A4310020C02800203A
:20830000F7B586B007460D463E200590002004902E4603970290002E03D11320344908706A
:2083200002E00020324908703148007800281AD1002405E00898005D2E490855601CC4B278
:20834000B442F7DB2B48007880210840C0090290284800784006400E04900498002802D080
:2083600012202349087022480078002804D1012E02D013201E4908701D48007800280BD114
:208380000298002832D11B4801231B4A00210090059800F033F829E017495631039888426E
:2083A0001CD113480078112820D01148007812281CD00F4800787E2818D00D4800787F280C
:2083C00014D00B480078312810D0094801230A4A19460090059800F011F807E00448012310
:2083E000054A19460090059800F008F809B0F0BD98020020C028002089070000FFB581B015
:20840000064617460A9D0298002822D0224807607F202149087108464671403104988884E7
:20842000002406E029781C48801D01556D1C601C84B219484030808CA042F3DC16494031A1
:20844000898C891C8AB214490868091DFEF710FF20E0124807604020304310490871403158
:2084600004988884002406E029780C48401D01556D1C601C84B209484030808CA042F3DCE9
:2084800006494031898C491C8AB204490868091DFEF7EEFE05B0F0BD58280020F027002069
:2084A00010B500200D4908700D4908700D4908700D4908700D480E49086000200D4908709D
:2084C0000D4908700D4908600D4908700D4908700D490870FBF764F910BD000096020020D2
:2084E00095020020940200209802002058D93401A00200209C0200209D020020A4020020EA
:20850000A80200209B0200209A02002070B504460D4629462046FEF75DFC70BD10B50548F4
:208520000078012805D10220FBF70CFC022000F009F810BDC0020020AC2001494870704761
:208540000010024070B588B005467D480068002821D07C48007800281ED10120794908702D
:20856000FF2281027848F8F72DFE78480068784A12688118744B012292020020FCF754FDA6
:20858000FF20F53073490880714800680121890240186F490860D1E000231A461946012059
:2085A000FCF742FD064669480068694909684118B14239D16848006800285AD1022DF8D148
:2085C00004AA1021654800F0C4FB10225E4910316846F8F7E5FD102204A95B481030F8F716
:2085E00003FE002833D058480830FAF73BF85A49086055480C30FAF735F8514908605648B1
:2086000000680321890388420FD14D4800681D218903884209D200205149086010204C4945
:20862000086000204749087076E0FAF781F84D4A51681068F9F7E6FE002802D100F098F8D3
:2086400002E0494800F094F8FEF7BCFD64E0FAF76FF8444A51681068F9F7D4FE002802D165
:2086600000F086F802E0404800F082F8FEF7AAFD52E03B48006832490968884230D23048CF
:20868000006837490968401A01218902884201D30C4604E02A48006831490968441A2A4A0F
:2086A00021462D48006800F0A8FA2B4800680019294908602A480068001929490860002029
:2086C00020490870022D27D1214909686422514308461B490968F8F739FD244908601BE085
:2086E000FAF726F81F4A51681068F9F78BFE00280DD100F03DF819491031184800F04AF9F7
:20870000032292031021154800F077FA02E0164800F02EF8FEF756FD0E480088401E80B2A4
:208720000C490880002809D10948006801218902401A0749086000200249087008B070BD1A
:2087400050000020780000206C130020580000205C0000207A0000206800002000185000F4
:2087600054000020BC310020A55AA55A6000002010B504460848094908600846446008499E
:208780000748083800F006F9044A08210448083800F033FA10BD0000A55A7AA7B402002078
:2087A0000810500030B47446641E2578641CAB4204D3635D5B00E31830BC18471D46F8E7AD
:2087C000002805DBC206D20E01219140014A11607047000080E200E010B5002819DB1A4AFC
:2087E00003231B02D21883089B00D2588307DC0EFF23A3409A438B071B0E8407E40EA3408B
:208800001A43114B032424021B198408A4001A5118E00E4A03071B0F083B9B089B00D25854
:208820008307DC0EFF23A3409A438B071B0E8407E40EA3401A43054B0407240F083CA408EC
:20884000A4001A5110BD000000E100E01CED00E002E008C8121F08C1002AFAD17047704783
:20886000002001E001C1121F002AFBD17047000010B502460EE01378521C094C24786340CF
:208880001B069B0D074CE358054C2468240A6340034C23600B46491E002BECD110BD000094
:2088A000AC020020908F000010B50021024841700248F9F773F810BD24600040005404401C
:2088C00010B500210D48417002210D48F9F7EAF8002812D002210A48F9F7B8F809490848A1
:2088E000F9F732FA0848FDF713FA08480068002803D0054805490968884710BD5C600040B4
:2089000000540440841700206C1700208000002070B5054600262C46202221461548F8F7C4
:2089200063FC002823D120222146403111484030F8F75AFC00281AD12022A1180D482030E1
:20894000F8F752FC002812D120222146603109486030F8F749FC002809D110222146803134
:2089600004488030F8F740FC002800D100E00126304670BD008F000010B5044603492046DD
:20898000F8F7E4FB0249087010BD000040420F009000002070B505460E462C460BE02046B1
:2089A00000F0E7F8A004800C002801D1FDF794F9012080022418B442F1D370BD70B5044608
:2089C000002C01D1064D01E0012070BD2846F9F740F8032801D10220F7E70020F5E7000088
:2089E0000054044072B60120000309498860BFF35F8F62B6F9F76AFDF9F7C4FDFDF796FD12
:208A0000FEF7F0FB03E0FDF767F9FDF711FDFAE700ED00E00346002B01D10B4A01E00120F2
:208A200070475020815A094801400720014350208152815A05480140FF2001300143502087
:208A400081520020ECE7000000540440F8F8000010B588B0044623231F2202210520FAF7C1
:208A60005BFF22231E2201210520FAF755FF02216846018300218176012181770021C176AC
:208A8000017706A90520FAF7A3FE01216846018381760021C17606A90520FAF799FE0421D4
:208AA0006846018300218176C176022141770021817706A90520FAF78BFE617868460170FB
:208AC00002214180002141710C2181710121C1710021017160680290A0680390E068049008
:208AE0002069059069460D48F9F700F80C496069086001210948F9F703F901220E210748E6
:208B0000F8F7DBFF07493720FCF766F806492920FCF762F8002008B010BD00000054044072
:208B200080000020C1880000A988000000BE00BFFEE77047014672B608208C4AD060F12054
:208B4000106255205060AA2090600020C043086000BF86480068C007C00F0028F9D001209C
:208B6000824A10600020D060F020106262B600207047014672B610207C4AD060F1201062E0
:208B800055205060AA2090600020C043086000BF76480068C007C00F0028F9D00120734A21
:208BA00010600020D060F020106262B60020704770B503461D46F1206C4E3062002415E03D
:208BC00072B6AA20694E70605520B06010782870521C6D1C62B600BF64480068C007C00FFF
:208BE0000028F9D00120614E3060641C8C42E7D3F0205E4E3062002070BDF7B55C4B9D444D
:208C000006460F4600215B4868448161012104918802874207D95748684481618069554BC1
:208C200028339D44F0BD029600240EE0029800785049694448610298401C02904869FF2840
:208C400001D000200490601C84B2BC42EED3049800280AD04848494908604648684439463D
:208C6000426A3046FFF7A4FF6FE0B00A4500F119681C4002814202D90120039001E00020C8
:208C80000390B10A89020191B105890D0091039800280ED0002408E00198007805A90855C3
:208CA0000198411C0191601C84B232488442F3DB0EE0002408E00198007805A908550198BD
:208CC000411C0191601C84B2012080028442F2DB002410E027486844406A027800990819B0
:208CE00005A90A5423486844406A411C214868444162601C84B2BC42ECD30398002815D07B
:208D00001D481E4908606802FFF733FF1A481B490860691C4802FFF72CFF17481749086048
:208D2000680205AA1349FFF743FF0EE01248134908606802FFF71DFF0F481049086068027C
:208D400005AA01218902FFF733FF0A486844806965E730B50446002304E025781570641C84
:208D6000521C5B1C8B42F8D330BD000000000240E4F7FFFF00080000CDAB341294000020F4
:208D800001020020FE0000FE000002020021FE0000FE000003020022FE0000FE000004026A
:208DA0000023FE0000FE00000502040AFE0000FE00000602001C020701FE00000702001D31
:208DC000FE0000FE000008020106020702FE000009020107020710FE00000A02010FFE0039
:208DE00000FE00000B02010EFE0000FE00000C020123FE0000FE00000D020423FE0000FEFD
:208E000000001002012EFE0000FE00001102012FFE0000FE00001202010F07041A07050A77
:208E20001302010E0704370705091402020CFE0000FE00001502020DFE0000FE000016025D
:208E40000319FE0000FE00000E02052BFE0000FE00000F02052AFE0000FE0000170400194E
:208E600004011B0408071804021E040301FE000019000029FE0000FE00001A000128FE00FE
:208E800000FE00001B00020E070909FE00001C000318FE0000FE00001D00041E07090CFE06
:208EA00000001E00051F07090BFE00002000060FFE0000FE00002107090AFE0000FE0000EF
:208EC0002207031EFE0000FE00002307031FFE0000FE000000FE0000FE0000FE0000010009
:208EE000020004000800100020004000800000010002000400080010002000400080000075
:208F0000484A5F3735305F5446540000000000000000000000000000000000000000000077
:208F2000484A59422D3735303054465400000000000000000000000000000000000000001D
:208F40004241543332413237394B4D36344642000000000000000000000000000000000068
:208F600043414E5F5354445F4348305F3530304B6270730000000000000000000000000037
:208F80008907000081070000DF0700000000000000000000963007772C610EEEBA51099959
:208FA00019C46D078FF46A7035A563E9A395649E3288DB0EA4B8DC791EE9D5E088D9D297C9
:208FC0002B4CB609BD7CB17E072DB8E7911DBF906410B71DF220B06A4871B9F3DE41BE84E9
:208FE0007DD4DA1AEBE4DD6D51B5D4F4C785D38356986C13C0A86B647AF962FDECC9658A89
:209000004F5C0114D96C0663633D0FFAF50D088DC8206E3B5E10694CE44160D5727167A2A8
:20902000D1E4033C47D4044BFD850DD26BB50AA5FAA8B5356C98B242D6C9BBDB40F9BCAC48
:20904000E36CD832755CDF45CF0DD6DC593DD1ABAC30D9263A00DE518051D7C81661D0BF68
:20906000B5F4B42123C4B3569995BACF0FA5BDB89EB802280888055FB2D90CC624E90BB108
:20908000877C6F2F114C6858AB1D61C13D2D66B69041DC760671DB01BC20D2982A10D5EFE8
:2090A0008985B1711FB5B606A5E4BF9F33D4B8E8A2C9077834F9000F8EA8099618980EE1C8
:2090C000BB0D6A7F2D3D6D08976C6491015C63E6F4516B6B62616C1CD83065854E0062F268
:2090E000ED95066C7BA5011BC1F4088257C40FF5C6D9B06550E9B712EAB8BE8B7C88B9FC88
:20910000DF1DDD62492DDA15F37CD38C654CD4FB5861B24DCE51B53A7400BCA3E230BBD427
:2091200041A5DF4AD795D83D6DC4D1A4FBF4D6D36AE96943FCD96E34468867ADD0B860DA47
:20914000732D0444E51D03335F4C0AAAC97C0DDD3C710550AA41022710100BBE86200CC9E7
:2091600025B56857B3856F2009D466B99FE461CE0EF9DE5E98C9D9292298D0B0B4A8D7C707
:20918000173DB359810DB42E3B5CBDB7AD6CBAC02083B8EDB6B3BF9A0CE2B6039AD2B1741F
:2091A0003947D5EAAF77D29D1526DB048316DC73120B63E3843B64943E6A6D0DA85A6A7AB7
:2091C0000BCF0EE49DFF099327AE000AB19E077D44930FF0D2A3088768F2011EFEC2066957
:2091E0005D5762F7CB67658071366C19E7066B6E761BD4FEE02BD3895A7ADA10CC4ADD6777
:209200006FDFB9F9F9EFBE8E43BEB717D58EB060E8A3D6D67E93D1A1C4C2D83852F2DF4F16
:20922000F167BBD16757BCA6DD06B53F4B36B248DA2B0DD84C1B0AAFF64A0336607A044136
:20924000C3EF60DF55DF67A8EF8E6E3179BE69468CB361CB1A8366BCA0D26F2536E26852D6
:2092600095770CCC03470BBBB91602222F260555BE3BBAC5280BBDB2925AB42B046AB35CF6
:20928000A7FFD7C231CFD0B58B9ED92C1DAEDE5BB0C2649B26F263EC9CA36A750A936D02D6
:2092A000A906099C3F360EEB8567077213570005824ABF95147AB8E2AE2BB17B381BB60CB6
:2092C0009B8ED2920DBED5E5B7EFDC7C21DFDB0BD4D2D38642E2D4F1F8B3DD686E83DA1FD6
:2092E000CD16BE815B26B9F6E177B06F7747B718E65A0888706A0FFFCA3B06665C0B011176
:20930000FF9E658F69AE62F8D3FF6B6145CF6C1678E20AA0EED20DD75483044EC2B3033995
:20932000612667A7F71660D04D476949DB776E3E4A6AD1AEDC5AD6D9660BDF40F03BD83735
:2093400053AEBCA9C59EBBDE7FCFB247E9FFB5301CF2BDBD8AC2BACA3093B353A6A3B42455
:209360000536D0BA9306D7CD2957DE54BF67D9232E7A66B3B84A61C4021B685D942B6F2AF5
:2093800037BE0BB4A18E0CC31BDF055A8DEF022D33373130302D433031312D3031303043E9
:2093A0003031312D56313030433031312D5631303020240723312E30345F3230323430385E
:2093C0003231000056312E3332203230323430353330000004940000000000201003000095
:2093E000241400003C94000000FF0020D0000000508800003C94000010030020685C0000D7
:2094000060880000018CB2C01AFF011133C14C09D00551890A890F09213209171E091723C3
:20942000012D0917A0092682091750091241014B0312C493EAFF10190101200040203149FB
:20944000087100BF00BF00BF00BF00BF2D480079802108400028F9D070471020294908713E
:2094600000BF00BF00BF00BF00BF26480079202108400028F9D0704723480078802108404D
:20948000002810D020480078400840001E49087000BF00BF00BF00BF00BF1B480078802146
:2094A00008400028F9D100201649087100BF00BF00BF00BF00BF13480079602108400028FA
:2094C000F9D1704710480078012108430E49087000BF00BF00BF00BF00BF0B4800788021D8
:2094E00008400028F9D000200649087100BF00BF00BF00BF00BF03480079402108400028FB
:0C950000F9D1704700040240000C02404A
:00000001FF
